:020000040000FA
:0600000027EF4BF0120097
:020006001200E6
:060008000FEF2EF01200C4
:02000E001200DE
:020010000100ED
:0500120000000000F6F3
:06001800B4EF18F0120025
:02001E000800D8
:10002000E1970000F908000004000000A19700001B
:100030009D0900004000000012000000F4080000CC
:10004000050000007C970000C807000025000000A4
:1000500047970000C8060000350000001097000018
:10006000C805000037000000B3960000000900003A
:100070005D00000010000000FE040000020000000F
:10008000FAEC0CF040EC0DF0EE6AEE6AEE6AEE6A05
:1000900073EC0CF0EE6AEE6AEE6AEE6AAFEC09F011
:1000A000010EEE6E230EEE6E450EEE6E670EEE6ED8
:1000B000AFEC09F0040EF1EC0AF0890EEE6EAB0E17
:1000C000EE6ECD0EEE6EEF0EEE6EAFEC09F0080E9A
:1000D000F1EC0AF0FE0EEE6EDC0EEE6EBA0EEE6E77
:1000E000980EEE6EAFEC09F00C0EF1EC0AF0760E05
:1000F000EE6E540EEE6E320EEE6E100EEE6EE55299
:10010000E7CFD9FF1200FAEC0CF0080EE126030E3F
:10011000046E73EC0CF025EC0BF003E045EC0BF0F7
:10012000FDE13F0E00167FEC0BF0B4EC0CF0F90E85
:10013000DBCF04F0FA0EDBCF05F0066A076A05AEE6
:1001400002D006680768030E1F0B07E0D89004363C
:10015000053606360736E806F9E173EC0CF0045074
:10016000EF26EECF00F00550EF22EECF01F0065063
:10017000EF22EECF02F00750EF22EECF03F0F90EA0
:10018000DBCF08F0FA0EDBCF09F00A6A0B6A09AE82
:1001900002D00A680B68030E1F0B03E056EC0BF04D
:1001A000FDE10850005C095001580A5002580B50FC
:1001B000035806E240EC0DF0EE2AEE22EE22EE228B
:1001C0005DEC0BF0026A036A01AE02D002680368BC
:1001D0001D0E45EC0BF0FDE140EC0DF0EDEC0CF0EC
:1001E000400E046E056A066A076AD9CFE9FF2BEC58
:1001F0000BF0EE500758060E00C0DBFF070E01C0E3
:10020000DBFF5DEC0BF017EC0DF001500318E8AECE
:1002100002D0033404D00250005C035001586AE35A
:10022000060EDBCFE6FF070EDBCFE6FF19EC0BF087
:10023000F6EC0CF0E9CF02F0EACF03F0DB50E92452
:10024000006E010EDB50EA2075EC0BF0DDEC3EF0A9
:10025000046E060EE15E0450F6EC0CF010EC0BF0B0
:10026000AFEC09F0E9CF02F0EACF03F034EC0BF089
:10027000060EDBCF28F0070EDBCF29F0040E28C0D6
:10028000DBFF050E29C0DBFF3F0EE76EDDEC0CF057
:10029000E7500026000E0122D6EC0CF001500318A6
:1002A000E8AE02D0033404D00250005C0350015881
:1002B0001EE2040EDBCF02F0050EDBCF03F0FB0ED7
:1002C000DB500224006EFC0EDB50032075EC0BF0BB
:1002D000AFEC09F0E9CF04F0EACF05F034EC0BF015
:1002E00033EC0DF0400EEE26000EED22CDD71EECC5
:1002F0000DF004D0040EDB6A050EDB6AD6EC0CF0C0
:10030000040EDB50025C006E050EDB50035875ECEA
:100310000BF04CEC0BF0046EFC0EDB500720056E6E
:1003200004C0E6FFE66EF6EC0CF0E9CF0AF0EACF87
:100330000BF0DB50E924086E010EDB50EA20096E59
:1003400008C0E6FFE66EDDEC3EF00C6E060EE15EE8
:100350000C50080EE15C02E2E16AE55220EF0BF07E
:100360006AEC0BF0080E3FEC0BF0100EF1EC0AF00B
:1003700010EC0BF0D9CFE6FFDACFE6FF64EC0BF020
:10038000030E046E25EC0DF0100EF1EC0AF025ECD6
:100390000BF003E045EC0BF0FDE13F0E00167FECA7
:1003A0000BF063EC0CF0380EEE5C000EEE58000E15
:1003B000EE58000EEE580DE2380E046E056A066A1D
:1003C000076A3CEC0DF02BEC0BF0026EEE50075878
:1003D00013D0780E086E096A0A6A0B6A3CEC0DF0BD
:1003E00084EC0DF0085C006EEE500958016EEE5082
:1003F0000A58026EEE500B58036E80EC0CF00C0E97
:10040000DBCFE6FF0D0EDBCFE6FF9D0EE66E090E9D
:10041000E66E19EC0BF06EEC0BF0080EE66EE66A79
:10042000D9CFE6FFDACFE6FF19EC0BF06EEC0BF05C
:10043000100E3FEC0BF010EC0BF0FD0EDBCFE6FFE7
:10044000FE0EDBCFE6FF64EC0BF0100EE15C02E287
:10045000E16AE55220EF0BF06AEC0BF0AFEC09F02B
:10046000EECFDFFF010EEECFDBFF020EEECFDBFFA4
:10047000030EEECFDBFF040E55EC0CF0040EEECFB6
:10048000DBFF050EEECFDBFF060EEECFDBFF070E28
:10049000EECFDBFF080E55EC0CF0080EEECFDBFFC5
:1004A000090EEECFDBFF0A0EEECFDBFF0B0EEECF19
:1004B000DBFF0C0E55EC0CF00C0EEECFDBFF0D0E3F
:1004C000EECFDBFF0E0EEECFDBFF0F0EEECFDBFF2E
:1004D000400EE66EE66AE66AE66A19EC0BF05D0E1F
:1004E000E66E090EE66E25EC08F0006E080EE15E81
:1004F0000050C9EC0BF010EC0AF0780E0026A40EA8
:1005000001226A0E0222D70EFFEC0CF003E055EC3C
:1005100009F0FDE127EC09F0190E44EC09F0FDE1CA
:1005200083EC0BF01DEC0AF0560E0026B70E0122EC
:10053000C70E0222E80E71EC0DF003E055EC09F055
:10054000FDE137EC09F0140E44EC09F0FDE19EECFE
:100550000BF02AEC0AF0DB0E0026700E0122200EB2
:100560000222240E44EC0DF003E055EC09F0FDE10D
:100570001AEC09F00F0E44EC09F0FDE1B6EC0BF0BB
:1005800037EC0AF0EE0E0026CE0E0122BD0E02223E
:10059000C10E75EC0DF003E055EC09F0FDE12AEC1D
:1005A00009F00A0E44EC09F0FDE179EC0DF044ECA1
:1005B0000AF0AF0E00260F0E01227C0E0222F50E6D
:1005C000FFEC0CF003E055EC09F0FDE127EC09F03D
:1005D000190E44EC09F0FDE183EC0BF051EC0AF04C
:1005E0002A0E0026C60E0122870E0222470E71EC4B
:1005F0000DF003E055EC09F0FDE137EC09F0140EC5
:1006000044EC09F0FDE19EEC0BF05EEC0AF0130EF9
:100610000026460E0122300E0222A80E44EC0DF0F8
:1006200003E055EC09F0FDE11AEC09F00F0E44EC83
:1006300009F0FDE1B6EC0BF06BEC0AF0002A950E28
:100640000122460E11EC0DF0160E1F0B03E055ECC7
:1006500009F0FDE12AEC09F00A0E44EC09F0FDE195
:1006600079EC0DF078EC0AF0D80E0026980E0122F5
:10067000800E0222690EFFEC0CF003E055EC09F04D
:10068000FDE127EC09F0190E44EC09F0FDE183ECE3
:100690000BF085EC0AF0AF0E0026F70E0122440E97
:1006A00002228B0E71EC0DF003E055EC09F0FDE138
:1006B00037EC09F0140E44EC09F0FDE19EEC0BF070
:1006C00092EC0AF0B10E00265B0E0122FF0E022210
:1006D00044EC0DF003E055EC09F0FDE11AEC09F0F3
:1006E0000F0E44EC09F0FDE1B6EC0BF09FEC0AF0C4
:1006F000BE0E0026D70E01225C0E0222890E75EC7A
:100700000DF003E055EC09F0FDE12AEC09F00A0ECA
:1007100044EC09F0FDE179EC0DF0ACEC0AF0220EAE
:100720000026110E0122900E02226B0EFFEC0CF03F
:1007300003E055EC09F0FDE127EC09F0190E44EC5B
:1007400009F0FDE183EC0BF0B9EC0AF0930E002602
:10075000710E0122980E7AEC0BF00C0FF4EC08F0FD
:1007600076EC09F00C0E1F0B03E055EC09F0FDE1EF
:1007700037EC09F0140E44EC09F0FDE19EEC0BF0AF
:10078000C6EC0AF08E0E0026430E0122790E0222DC
:10079000A60E44EC0DF003E055EC09F0FDE11AEC77
:1007A00009F00F0E44EC09F0FDE1B6EC0BF0D3ECD0
:1007B0000AF0210E0026080E0122B40E0222490E74
:1007C00075EC0DF003E055EC09F0FDE12AEC09F0C1
:1007D0000A0E44EC09F0FDE1EAEC0BF01DEC0AF026
:1007E000620E0026250E01221E0E0222F60E03ECDA
:1007F0000DF003E055EC09F0FDE127EC09F01B0ECC
:1008000044EC09F0FDE106EC0CF05EEC0AF0400E61
:100810000026B30E0122400E0222C00E48EC0DF05D
:1008200003E055EC09F0FDE137EC09F0170E44EC5C
:1008300009F0FDE1DDEC0BF09FEC0AF0510E002613
:100840005A0E01225E0E0222260E4CEC0DF003E041
:1008500055EC09F0FDE11AEC09F0120E44EC09F038
:10086000FDE1F2EC0BF010EC0AF0AA0E0026C70E28
:100870000122B60E0222E90E50EC0DF003E055EC19
:1008800009F0FDE12AEC09F00C0E44EC09F0FDE161
:10089000EAEC0BF051EC0AF05D0E0026100E01227E
:1008A0002F0E0222D60E03EC0DF003E055EC09F0FA
:1008B000FDE127EC09F01B0E44EC09F0FDE106EC2C
:1008C0000CF092EC0AF0530E0026140E0122440E96
:1008D0000222020E48EC0DF003E055EC09F0FDE1B8
:1008E00037EC09F0170E44EC09F0FDE1DDEC0BF0FC
:1008F000D3EC0AF0810E0026E60E0122A10E0222A0
:10090000D80E4CEC0DF003E055EC09F0FDE11AECCB
:1009100009F0120E44EC09F0FDE1F2EC0BF044ECAE
:100920000AF0C80E0026FB0E0122D30E0222E70EAB
:1009300050EC0DF003E055EC09F0FDE12AEC09F074
:100940000C0E44EC09F0FDE1EAEC0BF085EC0AF04A
:10095000E60E0026CD0E0122E10E0222210E03EC4E
:100960000DF003E055EC09F0FDE127EC09F01B0E5A
:1009700044EC09F0FDE106EC0CF0C6EC0AF0D60EF2
:100980000026070E0122370E0222C30E48EC0DF09E
:1009900003E055EC09F0FDE137EC09F0170E44ECEB
:1009A00009F0FDE1DDEC0BF037EC0AF0870E0026D4
:1009B0000D0E0122D50E0222F40E4CEC0DF003E0D8
:1009C00055EC09F0FDE11AEC09F0120E44EC09F0C7
:1009D000FDE1F2EC0BF078EC0AF0ED0E0026140EBF
:1009E00001225A0E0222450E50EC0DF003E055ECA8
:1009F00009F0FDE12AEC09F00C0E44EC09F0FDE1F0
:100A0000EAEC0BF0B9EC0AF0050E0026E90E012223
:100A1000E30E0222A90E03EC0DF003E055EC09F001
:100A2000FDE127EC09F01B0E44EC09F0FDE106ECBA
:100A30000CF02AEC0AF0F80E0026A30E0122EF0EAD
:100A40000222FC0E48EC0DF003E055EC09F0FDE14C
:100A500037EC09F0170E44EC09F0FDE1DDEC0BF08A
:100A60006BEC0AF0D90E0026020E01226F0E022254
:100A7000670E4CEC0DF003E055EC09F0FDE1DADB1C
:100A8000120E44EC09F0FDE1F2EC0BF0ACEC0AF0D4
:100A90008A0E00264C0E01222A0E02228D0E50ECE8
:100AA0000DF003E055EC09F0FDE1D4DB0C0EECDBBE
:100AB000FEE121EC0CF051EC0AF0420E0026390E5A
:100AC0000122FA0E0222FF0E07EC0DF002E0EDDB30
:100AD000FEE1BDDB1C0ED8DBFEE139EC0CF078EC5E
:100AE0000AF0810E0026F60E0122710E0222870EF8
:100AF00054EC0DF002E0D9DBFEE1B9DB150EC4DBEE
:100B0000FEE128EC0CF09FEC0AF0220E0026610EAC
:100B100001229D0E02226D0E58EC0DF002E0C5DBA5
:100B2000FEE188DB100EB0DBFEE141EC0CF0C6EC20
:100B30000AF00C0E0026380E0122E50E11EC0DF025
:100B4000170E1F0B02E0B1DBFEE184DB090E9CDB1C
:100B5000FEE121EC0CF01DEC0AF0440E0026EA0E3A
:100B60000122BE0E0222A40E07EC0DF002E09DDB76
:100B7000FEE16DDB1C0E88DBFEE139EC0CF044EC91
:100B80000AF0A90E0026CF0E0122DE0E02224B0E25
:100B900054EC0DF002E089DBFEE169DB150E74DB3D
:100BA000FEE128EC0CF06BEC0AF0600E00264B0E18
:100BB0000122BB0E0222F60E58EC0DF002E075DBAE
:100BC000FEE138DB100E60DBFEE141EC0CF092EC54
:100BD0000AF0700E0026BC0E0122BF0E0222BE0ECD
:100BE0007DEC0DF002E061DBFEE134DB090E4CDB55
:100BF000FEE121EC0CF0B9EC0AF0C60E00267E0EE8
:100C000001229B0E0222280E07EC0DF002E04DDBC4
:100C1000FEE11DDB1C0E38DBFEE139EC0CF010ECC4
:100C20000AF0FA0E0026270E0122A10E0222EA0E79
:100C300054EC0DF002E039DBFEE119DB150E24DB8C
:100C4000FEE128EC0CF037EC0AF0850E0026300EA1
:100C50000122EF0E0222D40E58EC0DF002E025DB4B
:100C6000FEE1E8DA100E10DBFEE141EC0CF05EEC88
:100C70000AF0050E00261D0E0122880E0222040E27
:100C80007DEC0DF002E011DBFEE1E4DA090EFCDAA6
:100C9000FEE121EC0CF085EC0AF0390E0026D00EB6
:100CA0000122D40E0222D90E07EC0DF002E0FDDA8B
:100CB000FEE1CDDA1C0EE8DAFEE139EC0CF0ACEC2A
:100CC0000AF0E50E0026990E0122DB0E0222E60E46
:100CD00054EC0DF002E0E9DAFEE1C9DA150ED4DADF
:100CE000FEE128EC0CF0D3EC0AF0F80E00267C0EA6
:100CF0000122A20E02221F0E58EC0DF002E0D5DAFE
:100D0000FEE198DA100EC0DAFEE141EC0CF0A2DB55
:100D1000650E0026560E0122AC0E0222C40E7DEC9A
:100D20000DF002E0C2DAFEE195DA090EADDAFEE17D
:100D30000FEC0CF075DB440E0026220E0122290E6A
:100D40000222F40E0CEC0DF002E0AFDAFEE17FDAE5
:100D50001A0E9ADAFEE1FAEC0BF0BDDB970E0026D4
:100D6000FF0E01222A0E0222430E5CEC0DF002E07F
:100D70009CDAFEE17CDA160E87DAFEE12FEC0CF04D
:100D8000C6EC0AF0A70E0026230E0122940E0222C2
:100D9000AB0E60EC0DF002E088DAFEE14BDA110EEA
:100DA00073DAFEE118EC0CF07CDB390E0026A00EA5
:100DB0000122930E0222FC0E64EC0DF002E075DAC3
:100DC000FEE148DA0B0E60DAFEE10FEC0CF0C4DB5A
:100DD000C30E0026590E01225B0E0222650E0CEC9A
:100DE0000DF002E062DAFEE132DA1A0E4DDAFEE1CF
:100DF000FAEC0BF03CDB920E0026CC0E01220C0E1E
:100E000002228F0E5CEC0DF002E04FDAFEE12FDAE9
:100E1000160E3ADAFEE12FEC0CF084DB7D0E002694
:100E2000F40E0122EF0E0222FF0E60EC0DF002E044
:100E30003CDAFEE1FFD9110E27DAFEE118EC0CF0E6
:100E4000FCDAD10E00265D0E0122840E0222850EF0
:100E500064EC0DF002E029DAFEE1FCD90B0E14DAA5
:100E6000FEE10FEC0CF044DB4F0E00267E0E01225B
:100E7000A80E02226F0E0CEC0DF002E016DAFEE175
:100E8000E6D91A0E01DAFEE1FAEC0BF08CDBE00E8B
:100E90000026E60E01222C0E0222FE0E5CEC0DF066
:100EA00002E003DAFEE1E3D9160EEED9FEE12FEC03
:100EB0000CF004DB140E0026430E0122010E022268
:100EC000A30E60EC0DF002E0F0D9FEE1B3D9110EF3
:100ED000DBD9FEE118EC0CF04CDBA10E0026110E64
:100EE0000122080E02224E0E64EC0DF002E0DDD964
:100EF000FEE1B0D90B0EC8D9FEE10FEC0CF0C4DA5C
:100F0000820E00267E0E0122530E0222F70E0CECFA
:100F10000DF002E0CAD9FEE19AD91A0EB5D9FEE168
:100F2000FAEC0BF00CDB350E0026F20E01223A0E25
:100F30000222BD0E5CEC0DF002E0B7D9FEE197D9BC
:100F4000160EA2D9FEE12FEC0CF084DABB0E0026BF
:100F5000D20E0122D70E02222A0E60EC0DF002E022
:100F6000A4D9FEE167D9110E8FD9FEE118EC0CF07F
:100F7000CCDA910E0026D30E0122860E0222EB0E51
:100F800064EC0DF002E091D9FEE164D90B0E7CD93E
:100F9000FEE10BD9E4D9C0EC0CF0040E55EC0CF0DA
:100FA000A7EC0CF0080E55EC0CF09AEC0CF00C0EC3
:100FB00055EC0CF08DEC0CF0100EE15C02E2E16AF5
:100FC000E5523ED312DBFCDA3AE2DFCF06F0010E47
:100FD000DBCF07F0D89006360736D89006360736AE
:100FE000FB0EDB50062413EC0DF00720EA6EEECF6B
:100FF00002F00250E66EDDEC0CF0B8D9080E44D9D0
:10100000FEE10450E66E010E49EC0CF0AFD9100E73
:101010003BD9FEE10450E66E020E49EC0CF0A6D975
:10102000180E32D9FEE10450E66E030E49EC0CF0C6
:1010300077EC0CF0E552E750EF6EE4DAC4D7080E17
:10104000E15C02E2E16AE552FBD2CFDAB9DA01E310
:10105000A2D022DB13EC0DF00720EA6EEFCF02F0F6
:10106000036A046A056A010E0C6E0D6A0E6A0F6A45
:1010700033EC0DF0EE500C26EE500D22EE500E2209
:10108000EE500F22FB0EDB500C2413EC0DF00D2064
:10109000EA6EEFCF08F0096A0A6A0B6A080E1F0BA6
:1010A00002E004DBFEE108500212095003120A506C
:1010B00004120B500512020E146E156A166A176A96
:1010C00033EC0DF0EE501426EE501522EE501622A1
:1010D000EE501722FB0EDB50142413EC0DF01520FC
:1010E000EA6EEFCF10F0116A126A136A100E1F0B2E
:1010F00007E0D8901036113612361336E806F9E1BB
:101100001050021211500312125004121350051203
:10111000030E1C6E1D6A1E6A1F6A33EC0DF0EE5042
:101120001C26EE501D22EE501E22EE501F22FB0EFA
:10113000DB501C2413EC0DF01D20EA6EEFCF18F0ED
:10114000196A1A6A1B6A180E1F0B07E0D890183626
:1011500019361A361B36E806F9E1185002121950F2
:1011600003121A5004121B500512DFCF00F0010EBB
:10117000DBCF01F0D89000360136D890003601362A
:10118000B6DB02C0EEFF03C0EEFF04C0EEFF05C0F9
:10119000EEFF38DA5BD7080EE15C02E2E16AE55265
:1011A0004FD288DB90DB8DEF0CF084DB040E00C0A7
:1011B000DBFF050E01C0DBFF060E02C0DBFF070EE2
:1011C00003C0DBFF33EC0DF09AEF0CF073DB98DB20
:1011D00068EC0DF0DACFEAFFC0EF0CF06BDBC4DB9C
:1011E00037EC0DF0A7EF0CF0E96EDACFEAFFEDEF88
:1011F0000CF0DACFEAFF0C50EE14086E0D50EE142E
:10120000096E0E50EE140A6E0F50EE140B6EC4D31E
:1012100003220050DE260150DE220250DE2203505F
:10122000DD22DD52DD5237EC0DF02CEC0DF0EFCF6E
:1012300003F01200080EDBCF04F0090EDBCF05F03F
:101240000A0EDBCF06F00B0EDBCF07F0120037ECF7
:101250000DF0BAD3040EDBCF04F0050EDBCF05F0A2
:10126000060EDBCF06F0070EDBCF07F012000C0EE8
:10127000DBCF04F00D0EDBCF05F00E0EDBCF06F05A
:101280000F0EDBCF07F01200D8900732063205327E
:101290000432E806120084EC0DF00816EE50091630
:1012A000EE500A16EE500B1677D3D8900036013662
:1012B00002360336E806120084EC0DF00416EE50F8
:1012C0000516EE500616EE5007161200DACFEAFFAA
:1012D0000850EE18046E0950EE18056E0A50EE180C
:1012E000066E0B50EE18076E045012000C0EDBCF8A
:1012F00000F00D0EDBCF01F00E0EDBCF02F00F0E73
:10130000DBCF03F01200080EDBCF00F0090EDBCFBD
:1013100001F00A0EDBCF02F00B0EDBCF03F0120060
:101320004CDB17EF0DF0F0DB041AEE50051AEE500F
:10133000061AEE50071A04501200E6DB081AEE50A7
:10134000091AEE500A1AEE500B1A1200DDDB0412D5
:10135000EE500512EE500612EE5007121200FD0E6E
:10136000DBCFE9FFFE0EDBCFEAFF1200C0DAE55269
:10137000E750EF6EDFCF08F0010EDBCF09F0D89019
:1013800008360936D89008360936FB0EDB5008249B
:101390004ADB0920EA6E18D30C0EDBCF08F00D0EE5
:1013A000DBCF09F00E0EDBCF0AF00F0EDBCF0BF018
:1013B0001200080EDBCF08F0090EDBCF09F00A0E91
:1013C000DBCF0AF00B0EDBCF0BF01200040EDBCFED
:1013D00008F0050EDBCF09F0060EDBCF0AF0070E92
:1013E000DBCF0BF0120043DBEECF08F0EECF09F0BD
:1013F000EECF0AF0EFCF0BF01200DBCF0FF00C1E98
:101400000D1E0E1E0F1E1200081E091E0A1E0B1EA8
:10141000D9501200041E051E061E071ED9501200C8
:1014200009015D25006E05505E21016E06505F21A9
:10143000026E07506021036E120009016125006EE3
:1014400005506221016E06506321026E075064212F
:10145000036E120009016525006E05506621016EBC
:1014600006506721026E07506821036E12000901C1
:101470006925006E05506A21016E06506B21026ECF
:1014800007506C21036E120009016D25006E055096
:101490006E21016E06506F21026E07507021036E9F
:1014A000120009017125006E05507221016E06506F
:1014B0007321026E07507421036E12000901752515
:1014C000006E05507621016E06507721026E07509E
:1014D0007821036E120009017925006E05507A21EA
:1014E000016E06507B21026E07507C21036E1200B4
:1014F00009017D25006E05507E21016E06507F2179
:10150000026E07508021036E120009018125006ED2
:1015100005508221016E06508321026E07508421FE
:10152000036E120009018525006E05508621016EAB
:1015300006508721026E07508821036E12000901B0
:101540008925006E05508A21016E06508B21026E9E
:1015500007508C21036E120009018D25006E055085
:101560008E21016E06508F21026E07509021036E6E
:10157000120009019125006E05509221016E06505E
:101580009321026E07509421036E120009019525E4
:10159000006E05509621016E06509721026E07508D
:1015A0009821036E120009019925006E05509A21B9
:1015B000016E06509B21026E07509C21036E1200A3
:1015C000F70EDBCF00F0F80EDBCF01F0EFD94BDAEE
:1015D0000050EE5C0150EE580250EE580350EE58A9
:1015E0001200E926000EEA22120004DA080EE126B3
:1015F00025DA040EDB6A050EDB6A060EDB6A070ECF
:10160000DB6A120034DAEE2A000EEE22EE22EE221F
:101610002ADA040EEE26000EEE22EE22EE22120050
:10162000E9CF00F0EACF01F0E9CFE6FFEACFE6FF2D
:101630001200FB0EDBCFE6FFFC0EDBCFE6FF120055
:10164000E16EE552E7CFD9FF120004501F0B04DA18
:10165000EECF03F0120058DA045C006EEE5005582D
:10166000016EEE5006581200E9CFE6FFEACFE6FF22
:101670002CEC02F0E552E552E552E5521200E66E1E
:10168000E66AE66AE66A25EF0DF0D8900332023288
:1016900001320032E8061200040EDBCF06F0050E20
:1016A000DBCF07F0FB0EDB5006241200D890083683
:1016B00009360A360B36E8061200F90EDBCF00F0C9
:1016C000FA0EDBCF01F012007DDC026E080EE15E47
:1016D000025012008FD9100EE126120083EC00F0A8
:1016E000006E060EE15E00501200016E00C0E6FFC3
:1016F000E66E12000222FD0E0322D9501200016A8A
:10170000026A036A12006ADDA5DDD9CFE9FFD4DDE4
:10171000AED9EECF0CF0EECF0DF0EECF0EF0EFCF56
:101720000FF00C1E0D1E0E1E0F1EA6D9F9EF08F0AD
:101730000322D950080F58DD83EF09F047DD87DD1C
:10174000C7D9BADD0C0EDBCF0CF00D0EDBCF0DF0E0
:101750000E0EDBCF0EF00F0E50DEDAD9F9EF08F0E7
:101760000322D9500C0F40DD76EF09F01ADD7FDD42
:1017700083D9A2DD080EDBCF0CF0090EDBCF0DF014
:101780000A0EDBCF0EF00B0E38DED9CFE9FFF9EFF2
:1017900008F050DDBDD990DD040EDBCF0CF0050E56
:1017A000DBCF0DF0060EDBCF0EF0070E26DE90D954
:1017B000F9EF08F00322D9508FD108DD4BDD88D92D
:1017C0007BDD04DE081E091E0A1E0B1ED9CFE9FFB1
:1017D0004BEF09F0EADC4BDD9BD96EDDDDDD14DE7D
:1017E000080F8FD1DEDC33DD47D966DDFCDD0CDE92
:1017F0000C0F87D1F3DC1EDD041E051E061E071E1E
:10180000D9CFE9FFA3DD84D993EF09F0E7DC12DD3E
:10181000D9CFE9FF51DDCDDDF7DD040F72D1C5DC95
:1018200026DDF8DD040FE96E91DD26D993EF09F08E
:10183000B8DC0DDDEFDD080FE96E88DD49D993EFE7
:1018400009F0B3DCB6DD64D978DD42D966EF09F082
:10185000BDDCC9DD3DD971DD5BD966EF09F0B6DCD1
:10186000F9DCD8DD0C0FE96E71DDD9CFE9FF93EF1C
:1018700009F0B4DCABDDD9CFE9FF5FDDFDD866EF61
:1018800009F08FDC89DDF8D858DDD9CFE9FF66EFA4
:1018900009F0006E34DFE7D8EE500026EE5001224A
:1018A000EE500222EE5003221200E76E58DDE750A0
:1018B000F1EF0AF004500012055001120650021216
:1018C000075003121200080E00C0DBFF090E01C012
:1018D000DBFF0A0E02C0DBFF0B0E03C0DBFFCCD820
:1018E000DACFEAFF12003BDD100EF1EF0AF0FD0E39
:1018F000DB500024E96EFE0EDB500120EA6E120080
:101900000C0E00C0DBFF0D0E01C0DBFF0E0E02C08F
:10191000DBFF0F0E03C0DBFF12000C0EDB50EE26C8
:101920000D0EDB50EE220E0EDB50EE220F0EDB50C2
:10193000EE221200080EDB50EE26090EDB50EE22DE
:101940000A0EDB50EE220B0EDB50EE221200040ECC
:10195000DB50EE26050EDB50EE22060EDB50EE22AB
:10196000070EDB50EE22120000C0DFFF010E01C0A7
:10197000DBFF020E02C0DBFF030E03C0DBFF120021
:10198000DF50EE26010EDB50EE22020EDB50EE227F
:10199000030EDB50EE22120008500412095005120B
:1019A0000A5006120B50071204501200F90EDBCF3A
:1019B00002F0FA0EDBCF03F01200040EDBCF00F0D2
:1019C000050EDBCF01F01200EECF04F0EECF05F0F4
:1019D000EECF06F0EFCF07F012000050EE260150D8
:1019E000EE220250EE220350EE221200B8DC180E56
:1019F000F1EF0AF0D9CFE6FFE1CFD9FF120008DC02
:101A0000070E1F0B120004DC050E1F0B120008EC62
:101A100009F0040E1F0B120008EC09F0060E1F0B54
:101A2000120068DE59D0E96EFC0EDB501200060E83
:101A3000DBCF02F0070EDBCF03F01200DE6ADE6AB6
:101A4000DE6ADD6ADD52DD521200FB0EDBCFE9FFFC
:101A5000FC0EDBCFEAFF1200EECF00F0EECF01F07C
:101A6000EECF02F0120054D8DACFEAFF1200D9CF3D
:101A7000E9FFDACFEAFF1200D950080FE96E120031
:101A800032DF040EF1EF0AF053DE110E1F0B1200CD
:101A900067DE090E1F0B12004BDE0E0E1F0B12002D
:101AA00089DE140E1F0B12005BDE0B0E1F0B1200E3
:101AB0003FDE100E1F0B120053DE0A0E1F0B12002A
:101AC00037DE0F0E1F0B120075DE150E1F0B1200F6
:101AD000D9500C0FE96E1200040FF4EC08F090EFEF
:101AE00009F03EDE0C0E1F0B120064DE160E1F0BFB
:101AF0001200D5EC08F0C9EF0BF05CDE170E1F0BDF
:101B00001200E96E4BEF09F0DACFEAFFEE50120057
:081B1000D950040FE96E120028
:081B18000601FB6BFC6B1200DF
:101B20000601CA6B12000601010ECB6F050E04EC14
:101B300017F00601BE0EFD6F6B0E4DEC17F00A0E8E
:101B400004EF17F00601BC0EFD6F6B0E4DEF17F0A2
:101B500068EC16F0030EE1260601FA0548E1450E91
:101B60000601055D44E0410E055D41E0610E055D45
:101B70003EE0670E055D3BE0500E055D38E0020E6D
:101B800005C6DBFF060EE66E060EE66E000EE66E7E
:101B9000050E18EC17F093EC16F0E3EC16F002E6E5
:101BA00059EC17F005E2FCEC17F0F7E3DB2AF5D768
:101BB00080EC18F0BCEC3FF016EC18F0000EE66E6E
:101BC000050E29EC16F0B40E006E6B0ED5EC17F076
:101BD000020EDBCF07F6080EE66E060EE66EBDECD3
:101BE00016F080EC18F07FEC37F01DEC17F078EC75
:101BF00018F0BCEC3FF016EC18F0DDEC16F0BDEC84
:101C000016F078EC18F071EC17F0B10EFD6F6B0E5A
:101C10004DEC17F0030EE15C02E2E16AE55241EFA0
:101C200016F068EC16F0050EE126D650016E006A3B
:101C3000030E00C0DBFF040E01C0DBFFD75022EC17
:101C400017F0DF6A080EDF5C0BE2DF50EA6AEE0F86
:101C5000E96E070EEA22EF5022EC17F0DF2AF2D7E6
:101C6000030EDBCFE6FF040EDBCFE6FF50EC44F0C3
:101C7000E552E552DF6A160EDF5C0DE26DEC16F000
:101C8000DF50EA6ACC0FE96E060EEA22E552E75011
:101C9000EF6EDF2AF0D70601E26B090E26EC18F092
:101CA000D80EE66E040EE66E3FEC17F0BCEC3FF08B
:101CB00043EC16F03FEC17F0160EE66EE66A5EECAB
:101CC00017F020EC47F0026E0A0EE15E02500601AA
:101CD000A90EFD6F6B0E4DEC17F05EEC17F012ECD9
:101CE00017F0A70EFD6F6B0E4DEC17F0EEEC16F033
:101CF00071EC17F0A70EFD6F6B0E4DEC17F0080E90
:101D000026EC18F03FEC17F012EC17F0B10EFD6F57
:101D10006B0E4DEC17F0050EE15C02E2E16AE55254
:101D200041EF16F022EC18F0A00E006E6B0ED5EC11
:101D300017F03EEC18F009010551E66EE66A03C99A
:101D4000E6FF04C9E6FFBDEC16F063EC17F0930E56
:101D5000006E6B0E09EC16F00D0EE15E0350F9EC0F
:101D600015F0090109510F0A18E0020A12E0090AE8
:101D70000CE0060A06E0030A14E1890E006E6B0E01
:101D800013D0810E006E6B0E0FD07B0E006E6B0EAB
:101D90000BD0720E006E6B0E07D0690E006E6B0ECC
:101DA00003D0600E006E6B0E7DEC18F009010B5134
:101DB000040A12E0070A0CE0020A06E0010A10E138
:101DC000560E006E6B0E0FD04D0E006E6B0E0BD0CC
:101DD000460E006E6B0E07D0390E006E6B0E03D0F0
:101DE000370E006E6B0E7DEC18F088EC16F04D0887
:101DF0000AE114C9E6FF15C9E6FF330E006E6B0E4B
:101E000009EC18F00AD014C900F015C901F0040E4D
:101E1000A4EC17F0FDE1A3EC18F0F9EC15F088EC58
:101E200016F04D080AE116C9E6FF17C9E6FF330EA2
:101E3000006E6B0E09EC18F00AD016C900F017C935
:101E400001F0040EA4EC17F0FDE1A3EC18F0F9EC9E
:101E500015F058C900F0016A00BE016804EC18F0E2
:101E600051C9E6FF52C9E6FF50C902F0036A02BE3B
:101E7000036802C0E6FF03C0E6FF09010B51E66EEE
:101E8000E66A09010951E66EE66A09010A51E66E41
:101E9000E66A09010D51E66EE66A09010C51E66E2B
:101EA000E66A07C9E6FF08C9E6FF09010651E66EC2
:101EB000E66A150E046E6B0E056E066A04C0E6FF38
:101EC000E66E06C0E6FFF4EC17F0076E190EE15E51
:101ED000075085EC18F0020EE15C02E2E16AE5527F
:101EE00041EF16F00E0E006E6B0ED5EC17F0B7EC4E
:101EF00017F056C900F0016A00BE0168F6EC16F052
:101F0000010E026E6B0EFFEC15F00D0EE15E05503A
:101F100085EF18F068EC16F0090EE126090136513C
:101F200007E1375105E1385103E1395101E18AD028
:101F3000FA0E006E6A0ED5EC17F0DF6A040EDF5C55
:101F400073E288EC17F0EFCF00F0000EE76E001898
:101F5000E8AE02D0003403D0E750D88000545DE2F0
:101F6000DF50EA6A3A0FE96E090EEA22EFCF04F079
:101F700004C029F056EC3CF027C000F028C001F066
:101F800029C002F02AC003F0560E2C6E0E0E2D6EE4
:101F90008D0E2E6E3E0E2F6E82EC3CF0D4EC3DF09A
:101FA000010E26C0DBFF020E27C0DBFF030E28C098
:101FB000DBFF040E29C0DBFFCAEC16F0050E26C0BD
:101FC000DBFF060E27C0DBFFCAEC16F0070E22C0AF
:101FD000DBFF080E23C0DBFF88EC17F0EF50D80FB3
:101FE000006E016A00BE016804EC18F0070EDBCF3A
:101FF000E6FF080EDBCFE6FF050EDBCFE6FF060EA1
:10200000DBCFE6FFF00E026E6A0EFFEC15F00B0E52
:10201000E15E0550F9EC15F005D0EB0E006E6A0E8E
:102020007DEC18F0DF2A8AD757C900F0016A00BE9C
:10203000016804EC18F0E80E026E6A0E0EEC18F05F
:1020400085EC18F0090EE15C02E2E16AE55241EF2D
:1020500016F0E10E006E6A0ED5EC17F0C70EE66EB4
:10206000080EE66E0801DB51E66EE66A09015C5176
:10207000E66EE66A210EE66E090EE66E0901025171
:10208000E66EE66A0151E66EE66A0051E66EE66AC1
:10209000CC0E006E6A0E09EC16F0130EE15E0350D2
:1020A00085EF18F068EC16F0040EE12609011C51CA
:1020B0001D111E111F1107E1DE6ADE6ADE6ADD6A8C
:1020C000DD52DD521CD01C0EE96E090EEA6EEE5098
:1020D0000901185D006EEE501959016EEE501A5943
:1020E000026EEE501B59036E00C0DFFF010E01C0EF
:1020F000DBFF020E02C0DBFF030E03C0DBFFC50ED9
:10210000006E6A0ED5EC17F054C900F0016A00BEEB
:10211000016804EC18F055C902F0036A02BE0368B6
:1021200002C0E6FF03C0E6FF09011051E66EE66A51
:1021300020C904F0056A04BE056804C0E6FF05C0B6
:10214000E6FF68EC17F0EECFE6FFEECFE6FFEECF4E
:10215000E6FFEFCFE6FF09011251E66EE66A40C9DD
:10216000E6FF41C9E6FF42C9E6FF43C9E6FF3EC9B3
:10217000E6FF3FC9E6FF35C906F0076A06BE0768F5
:1021800006C0E6FF07C0E6FF34C908F0096A08BECA
:10219000096808C0E6FF09C0E6FF33C90AF00B6A08
:1021A0000ABE0B680AC0E6FF0BC0E6FF0901115129
:1021B000E66EE66A09010F51E66EE66A09010E5104
:1021C000E66EE66A990E0C6E6A0E0D6E0E6A0CC013
:1021D000E6FFE66E0EC0E6FFF4EC17F00F6E250E7C
:1021E000E15E0F5085EC18F0040EE15C02E2E16A5A
:1021F000E55241EF16F068EC16F0920E006E6A0E92
:10220000D5EC17F056C900F0016A00BE0168F6EC83
:1022100016F009011251E66EE66A63EC17F022EC43
:1022200016F07C0E026E6A0EFFEC15F0130EE15EE6
:102230000550F9EC15F0B7EC17F08ADC6FEF18F0E9
:1022400068EC16F0060E8FEC17F088EC16F009E03B
:1022500088EC16F0200805E0DF2A010EF6E3DB2A01
:10226000F4D788EC16F0200801E0C7D096EC17F000
:1022700001E3DB2AEF6A22EC16F05EEC17F076EC55
:1022800017F001E1BAD0090EE66E9EEC16F0D80EFA
:10229000E66E040EE5EC17F022EC16F0A8EC16F052
:1022A00022EC16F046EC17F078EC18F0EEEC16F095
:1022B0007FEC37F01DEC17F078EC18F0BDEC16F061
:1022C00076EC17F001E099D022EC16F0000EE66EE5
:1022D000060E18EC17F05EEC17F0D0EC17F0D80EE5
:1022E000E66E040EE5EC17F078EC18F0A8EC16F0AA
:1022F00078EC18F046EC17F0EEEC16F045EC18F020
:102300002EEC17F009EC17F002E659EC17F00AE290
:102310009DEC18F0E0EC16F0040EDB2A050EF2E35B
:10232000DB2AF0D7EEEC16F04DEC18F02EEC17F09F
:1023300009EC17F002E659EC17F00AE29DEC18F0F0
:10234000DDEC16F0040EDB2A050EF2E3DB2AF0D7F3
:102350000601010ECA6F0A0EE66E9EEC16F0FCEC4A
:1023600015F0500848E10601FA5123E1040EDB6A3A
:10237000050EDB6A09EC17F004E6160E005C000E91
:10238000015815E26DEC16F0040EDBCFE9FF050EE7
:10239000DBCFEAFFE30EE926060EEA22E552E7501C
:1023A000EF6E040EDB2A050EE5E3DB2AE3D7060118
:1023B000F96BFA6B740E006E6A0ED5EC17F0A9EC8F
:1023C00017F0D0EC17F093EC0DF06DEC17F0060160
:1023D000010EFA6FE66E9EEC16F0E80EE66E040E45
:1023E000E5EC17F0A9EC17F0A8EC16F0A9EC17F043
:1023F00046EC17F002D00601FA6B060EE15C02E231
:10240000E16AE55241EF16F022EC18F00601CA51DC
:1024100014E1070EE66EE66A6C0E006E6A0ED8ECEA
:1024200017F022EC16F07BEC17F001E0A6D0070EB7
:102430005BEC16F005DFE5521CD08DEC18F078EC63
:1024400018F022EC16F03BEC38F0E552E55216ECB1
:1024500018F0E0EC16F0050EE66EE66A660E006E09
:102460006A0EC4DB7BEC17F006E0400EE66E43EC30
:102470001AF0E55282D0D950FD0FE96EDACFEAFFAB
:10248000050EEE6E060EED6EE7EC16F0EF50450809
:102490003DE155EC18F04D0839E1D950FD0FE96EDA
:1024A000FF0EDA20EA6E020EEE26000EED228DEC13
:1024B00018F0010EE66E050EE66E010E5BEC16F0EE
:1024C0003BEC38F088EC18F0C5EC16F093EC16F005
:1024D000E3EC16F002E659EC17F005E2FCEC17F01D
:1024E000F7E3DB2AF5D7BDEC16F0010EE66E050E1C
:1024F000B0DBE7EC16F0EFCF00F5D950FD0FE96E39
:10250000DACFEAFF000EEE6E050EED6EE7EC16F088
:10251000EF50430A29E0190A0FE01B0A2EE15F0E73
:10252000006E6A0ED5EC17F00601CB5126E193EC54
:102530000DF0A8EC0DF012D055EC18F0300811E0B9
:102540000901010E5B6F0601CB5117E193EC0DF011
:1025500092EC0EF0C7DCDEDC7CDDA4DDA2EC0DF03D
:102560000CD009015B6B09D0010EA5DB0CD8E5523C
:10257000E5520601CB5101E130D8020EE15C02E2E6
:10258000E16AE5527ED3A4DB040E8FEC17F0C0DBCA
:1025900008E0BEDB2C0805E0DF2A010EF8E3DB2AA9
:1025A000F6D7B6DB2C0805E196EC17F001E3DB2A41
:1025B000EF6A48DB32EC18F0F3CFFBF6F4CFFCF611
:1025C000BDEC16F0600EE66E000E18EC17F0040E6F
:1025D000E15C02E2E16AE55254D37ADB040EE126C3
:1025E000020E04EC17F0280E0601FCAF02D0D890C2
:1025F00003D0FB5D000EFC5907E3FC3507E2FB51FD
:102600003108000EFC5502E293EC0DF0310E06018C
:10261000FB1901E1FC5101E118D2290EFB1901E17E
:10262000FC5101E107D2280EFB1901E1FC5101E147
:10263000E0D1180EFB1901E1FC5101E1CCD1170EDC
:10264000FB1901E1FC5101E1B0D1160EFB1901E1CA
:10265000FC5101E1A4D1150EFB1901E1FC5101E18E
:1026600098D1140EFB1901E1FC5101E18CD1130E3C
:10267000FB1901E1FC5101E180D1120EFB1901E1CE
:10268000FC5101E174D1110EFB1901E1FC5101E192
:102690004DD1100EFB1901E1FC5101E12AD10F0EC1
:1026A000FB1901E1FC5101E11ED10C0EFB1901E106
:1026B000FC5101E108D10B0EFB1901E1FC5101E1D4
:1026C000EED00A0EFB1901E1FC5101E1E0D0050E4C
:1026D000FB1901E1FC5101E1D2D0040EFB1901E12B
:1026E000FC5101E196D0030EFB1901E1FC516EE0B3
:1026F000020EFB1901E1FC5121E0010EFB1901E082
:10270000B3D1FC5101E0B0D1DE6ADD6A5CDB04E6E6
:10271000100E005C000E015801E3AED1C1DBEF509A
:10272000E66EE66A100EE66EE66A27DB4C0E006E79
:102730006A0E5CDA99DBEAE3DB2AE8D7B2DA5CDA24
:1027400008E013EC18F005E0B3EC17F0F8E3DB2A2F
:10275000F6D713EC18F001E005D107DB01E3DB2A23
:102760005BEC18F001E086D0E8DB04E6100E025CBA
:10277000000E035801E37ED057DA32EC18F0F35024
:10278000E66E8EDBE552E750EF6E1DDB04E6080EC9
:10279000005C000E01580FE347DA73EC18F0080EE6
:1027A000005E000E015A180E0024E66EB4EC44F0F0
:1027B000E552E552E5528CDB0F0EEE1801E017D121
:1027C000ED5001E014D15EEC2EF011D1DE6ADD6A2D
:1027D000FADA04E6200E005C000E015801E34CD149
:1027E000DFCFE6FFABDA74DB090EEE1805E1ED5042
:1027F00003E168EC18F0EF6A17DA200EE66EE66A7D
:10280000BCDA390E006E6A0EF1D92EDBE1E3DB2A69
:10281000DFD747DAF1D907E013EC18F004E0A3DBC7
:10282000F9E3DB2AF7D713EC18F001E09BD09DDA2F
:1028300001E3DB2A5BEC18F01DE17FDB04E6180EF8
:10284000025C000E035816E2EFD9DFCFE6FFB4ECCE
:1028500044F0E552E552E552CADBC8D9ECDB38DB7F
:10286000020EEE1801E006D1ED5001E003D15EEC5E
:102870002EF000D153DA810E006E910EF9D0B7DB45
:10288000B5D980DA040EE66E43EC1AF0EBD00801FD
:10289000DB5101E1A3D0EBDB53EC32F0A7D0080110
:1028A000DB5101E19BD0040E09010E1507E0070E74
:1028B00009010A5D03E0010EE66E0DD02FDAA30ECA
:1028C000006E910ED5D00801DB5101E187D00901DE
:1028D0000EA904D0E66A67EC32F088D01FDAD10E78
:1028E000006E910EC5D00801DB5101E177D068DBA5
:1028F00017D00801DB5172E0D4D97ED906E093DB12
:1029000004E031DBFAE3DB2AF8D78DDB2BE12DDAAB
:1029100001E3DB2AEF6AABDB53EC32F0E55284D9FA
:10292000A1DBF350E66E5DEC32F060D00801DB51C4
:1029300055E0B7D961D906E076DB04E014DBFAE3B1
:10294000DB2AF8D770DB0EE110DA01E3DB2AEF6A4D
:102950006BD930EC43F097D98ADBE2EC32F0E552E8
:10296000E55244D0DBD9450E006E910E81D00801AE
:10297000DB5134E032EC32F03AD00801DB512EE08A
:102980003FEC32F034D00801DB5112E019DB020ECB
:1029900016D00801DB510CE013DBE66A11D0080108
:1029A000DB5106E00DDB030E0AD00801DB5105E127
:1029B000B5D95F0E006E910E09D002DB010EE66EF6
:1029C00071EC32F0E552E552E55211DB47DB1CDADF
:1029D00052EC10F051D00801DB5105E19FD95F0E98
:1029E000006E910E45D043DB09EC33F0E552FFDA7F
:1029F0003FD057D901D906E016DB04E0B4DAFAE398
:102A0000DB2AF8D710DB0FE1B0D901E3DB2AEF6A4C
:102A1000D7DAC0EC20F0E552E55206D903DABC0E55
:102A2000FD6F6B0E17D093EC0DF078D9450E006E4C
:102A3000910E14D006012D0EFD6F6A0E2EDAC0DA4B
:102A4000F1D9270EFD6F6A0E05D0BADAEBD9250E43
:102A5000FD6F6A0E22DA050E0EDBC9DAFFDAE66ECA
:102A6000EDEC41F0E55208D059D91A0E006E6A0E0D
:102A7000BDD8E1DAA8EC0DF0A2EC0DF00601FB6B7D
:102A8000FC6B0001606B040EE15C02E2E16AE5525E
:102A9000F8D01ED90601CA5121E0CB5100081EE32F
:102AA000020E57DB070E006E6A0E27DBCBD878DAF2
:102AB000FE0E006E690E21DBAA0EE76EFB0EDBCF69
:102AC000E9FFFC0EDBCFEAFF49DAEF6AFB0EDBCF52
:102AD000E6FFFC0EDBCFE6FF63DAFFD900D3B2DA04
:102AE00038DB09010B51040A12E0070A0CE0020A64
:102AF00006E0010A10E1F20E006E690E0BD0E70E3F
:102B0000006E690E07D0DE0E006E690E03D0CF0E88
:102B1000006E690EF2DA090109510F0A18E0020A83
:102B200012E0090A0CE0060A06E0030A14E1C60EE8
:102B3000006E690E13D0B00E006E690E0FD0A20E9B
:102B4000006E690E0BD0980E006E690E07D0860ECF
:102B5000006E690E03D0750E006E690ECEDA660E39
:102B6000006E690ECADA8ADAD3D84D0809E114C9B1
:102B7000E6FF15C9E6FF600E006E690E4ADA0CD05A
:102B800014C900F015C901F0040EDED9FEE163D8C6
:102B90005A0E026E690E42DA2CD8530E006E690E80
:102BA000ACDA91D94E0E006E690E33DA22D895D97F
:102BB000020EE15C02E2E16AE55263D043DA5BDADD
:102BC000230E006E690EF1D988D9020EE15C02E293
:102BD000E16AE55256D036DA76D9EA0E006E680E12
:102BE0003DDAE15C02E2E16AE5524BD0E1D978EFEF
:102BF00018F086DAD0EF17F06BDAEF501200036EA0
:102C0000046A02C0E6FFE66E04C0E6FFEDD9056E79
:102C10001200CED9E9D9036E120046EC3FF0036EE4
:102C2000050EE15E03501200020EDBCFE6FF030E3D
:102C3000DBCFE6FF1200A3EC3FF0036E050EE15E72
:102C400003501200FD0EDBCFE6FFFE0EDBCFE6FFEA
:102C500012006ADAC1D1050E0026000E01220A0E0A
:102C60002D6E2E6A00C028F001C029F0DFEC4AF07A
:102C700028C000F029C001F028C0E6FF29C0E6FF07
:102C80001200E16E2CD2E552E552F3CF00F0F4CF02
:102C900001F0F3CFE6FFF4CFE6FF120091D932EF57
:102CA00018F0D950020FE96EDACFEAFF600EEE6E2F
:102CB000000EED6E1200E76EFD0EDBCF00F0FE0E93
:102CC000DBCF01F0E7500026000E012204EF18F0E0
:102CD000D9CFE6FFE1CFD9FF120057EC44F0F3CF94
:102CE000F6FFF4CFF7FF400E2D6E2E6AF6CF28F0D8
:102CF000F7CF29F05CEC3DF024C0F6FF25C0F7FFCC
:102D0000F00EF626930EF7220800F550E66E12003C
:102D1000DECFE9FFDDCFEAFFEF501200FBC6E6FF92
:102D2000FCC6E6FF1200100EE66EE66AE80EE66EDE
:102D3000040EFAD9C5D9DE6ADD6A12006FEC44F0E0
:102D4000E552020EF3CFDBFF030EF4CFDBFF1200E0
:102D5000BCEC3FF0E552E552F3CF02F0F4CF03F0C4
:102D6000F3CFE6FFF4CFE6FF1200020EDBCFE9FF60
:102D7000DB2A030EDBCFEAFF1200DECFE6FFDDCF5A
:102D8000E6FF120058D9A8EF0DF0F3CFDEFFF4CF25
:102D9000DDFF1200010EDBCF26F0020EDBCF27F0A5
:102DA000030EDBCF28F0040EDBCF29F00A0E2B6ECA
:102DB0002C6A2D6A2E6A82EF3DF09AD96ED90CD119
:102DC00097D963D909D18FD9D89001501200FD0E3F
:102DD000DBCFE9FFFE0EDBCFEAFF1200100EE66E3E
:102DE000E66AD80EE66E040EE66E12000DD90901F1
:102DF0005351E66EE66A4EC9E6FF4FC9E6FF4CC97D
:102E0000E6FF4DC9E6FF1200E66EEDEC41F0E5523B
:102E10001200040EDBCF00F0050EDBCF01F0D890DE
:102E200001501200FAEC19F0E552E55206011200C9
:102E3000E66E82EC3FF088EF18F0006E060EE15E61
:102E400000501200006E016AD950030FE96EDACF0C
:102E5000EAFF0050EE260150ED22120031D9040E97
:102E6000DB6A050EDB6A120004EC49F0036E0B0E00
:102E7000E15E0350A8EC0DF0DF2A010E1200010EF6
:102E8000DBCFE6FF020EDBCFE6FF120020EC47F0BF
:102E9000046E0A0EE15E04501200FE6FE8EF19F0B6
:102EA000DECFE9FFDDCFEAFFCC0EE926080EEA22ED
:102EB0001200000E005C040E01581200CC0EE66EEB
:102EC000060EE66E120009011351E66EE66A120064
:102ED000D9CFE9FFDACFEAFF1200A8EC0DF0A2EF9C
:102EE0000DF0D4EC37F014D90601120062EC3FF07B
:102EF0000FD900091200BEEC3EF0036E070EE15E32
:102F0000035000091200EFD80001800E01141200D6
:102F1000DF50EA6A360FE96E090EEA221200E12656
:102F2000FD0EDBCFDEFFDBCFDDFF1200DFCFE9FFE1
:102F3000DF2A010EDBCFEAFF1200DECF02F0DDCF89
:102F400003F0D89003501200D89000360136E80400
:102F50001200E30EE66E060EE66E1200E750E9265A
:102F6000000EEA221200020EDB2A030E1200C8D85D
:102F700044C9E6FF45C9E6FF46C9E6FF47C9E6FF83
:102F8000EED8370E006E6B0EB8D8BAD848C9E6FF37
:102F900049C9E6FF4AC9E6FF4BC9E6FFAFEF18F0A3
:102FA000A7D822EC3FF088EF18F020DE1BEF16F0D8
:102FB000016E026A00C0E6FFE66E02C0E6FF120084
:102FC000600EE66E000EE66E1200E66E2DDEBCECC4
:102FD0003FF059DE14EF16F0E66E29EC41F0006E7A
:102FE000080EE15E005012008BD804EF49F096DE27
:102FF0003A0E006E910E1200A0D8000EE66E060E7C
:1030000028DEDF2A010E120000C0E6FF01C0E6FF45
:103010001200FFDD070EE15E03501200F0DD070E27
:10302000E15E05501200E8DD2C081200E552E55281
:10303000ACDEBDEF16F004EC49F0036E070EE15E66
:103040000350120045DE020EE1261200E66E6FEC20
:1030500044F0E552DE5299DEDD521200C7DD92DE09
:10306000020E120030EC43F0E552E552120016DE7B
:10307000F350E66E1200C8DE93EF0DF0020EE66E1E
:103080006FEC44F0E552C5EF16F0000EE66E020E4E
:10309000E66EFA0EE66E040E1200000EE66E010EEB
:1030A000E66EF80EE66E040E1200010EE76E8FDE7D
:1030B00055DFEF501200EF6AF1DD67DE83EF17F0A6
:1030C000E66E80EC40F0006E080EE15E00501200EB
:1030D000020EDBCFE9FF030EDBCFEAFF1200E55261
:1030E000E7CFD9FF1200DECF00F0DDCF01F01200F4
:1030F000000EE66E060EE66E120078DD0DEF16F09D
:10310000000EE66E050EE66E120073DDA8EF0DF000
:10311000E552E552E552E5521200B10E006E6B0E1B
:1031200047DF90DD0DEF16F0E66E000EE66E030E43
:10313000E66EFC0EE66E040E12000601006B010E38
:10314000E66EE66A120087DD330E026E6B0E0EEF3E
:1031500018F091DF120E006E6A0ED5EF17F00BEC2F
:0831600042F06BDEF9EF15F0FF
:08316800D8CFE4FFE0CFE4FF43
:10317000E46EDACFE4FFE2CFDAFFE9CFE4FFEACF93
:10318000E4FFF6CFE4FFF7CFE4FFF5CFE4FFF3CFA2
:10319000E4FFF4CFE4FFFACFE4FF00EE20F0140EDA
:1031A000E80403E3EECFE4FFFBD700EE00F0200ECF
:1031B000E80403E3EECFE4FFFBD7E652B3EC46F0BE
:1031C00012EC48F0E55200EE1FF0200EE80403E395
:1031D000E5CFEDFFFBD700EE33F0140EE80403E378
:1031E000E5CFEDFFFBD7E5CFFAFFE5CFF4FFE5CF65
:1031F000F3FFE5CFF5FFE5CFF7FFE5CFF6FFE5CF2E
:10320000EAFFE5CFE9FFE5CFDAFFE550E5CFE0FFE4
:10321000E5CFD8FF10000801009B120084EC20F0DD
:10322000E652D9CFE6FFDACFE6FF89EC46F0E55269
:10323000E552000901E1C9D0FF0E0701E85D01E098
:1032400088D00D0EDF5CEDE089EC20F03CEC20F046
:1032500003E1015001E1E7073A0EDF5C1EE1060ED3
:10326000E75D1BE360EC20F018E1490E015D15E11C
:10327000500E025D12E1440E035D0FE10701E70508
:10328000CCEC1FF0EF6A050EE66E070EE66E22EC40
:1032900020F0FD0EE86FE76BC4D70A0EDF5CC1E1DA
:1032A0000701E707A9EC20F0040EE75D70E360EC8E
:1032B00020F06DE1430E015D6AE14D0E025D67E1B4
:1032C000540E035D64E1070EDF6EDF50DF2ACCECA5
:1032D0001FF0EF50220804E00701E751DF5CF5E33F
:1032E000DF04CCEC1FF0EF6A0701D36B140EE66E1F
:1032F000E66A070EE66E070EE66ED30EE66E070E62
:10330000E66E1AEC40F0006E060EE15E005007011A
:10331000E66BE7C7DFFFDF50DF06CCEC1FF0EF50B6
:103320002C0803E0DF500008F6E3DF50016A000FCD
:10333000006E070E0122020E0026000E012200C0C0
:10334000E6FF01C0E6FF22EC20F0E76BFE0EE86F1F
:1033500068D7FE0EE85D1EE10D0EDF5C03E00A0E8D
:10336000DF5C07E1E751E72BCCEC1FF0200EEF6E9E
:1033700002D089EC20F03CEC20F003E1015001E1A7
:10338000E707E907E95101E04CD7A9EC20F065D93E
:10339000070118D00D0EDF5C08E089EC20F03CEC52
:1033A00020F003E1015001E1E707E9070A0EDF5CC5
:1033B00006E1E707A9EC20F050D90701E76BE951D6
:1033C00001E02FD7E76BE8692CD7E552FDEF1FF03E
:1033D00059EC20F00EE0080100B1FDD759EC20F0C7
:1033E000E66E62EC46F0E5520601FD2B000EFE2370
:1033F000EFD7120084EC20F04DEC20F00FE0080134
:1034000000B1FDD74DEC20F0E66E62EC46F0E552DF
:10341000FD0EDB2AFE0EF0E3DB2AEED7FDEF1FF0F8
:1034200084EC20F0080100B1FDD7FE0EDBCFE6FFF3
:1034300062EC46F0E552FDEF1FF084EC20F0040E44
:10344000E126030EE66E7CEC20F0E60E026E680EBE
:10345000D2EC1FF003E0FE0EDBCFC8F5E30E026EE8
:10346000680ED2EC1FF003E0FE0EDBCFC8F6040EB0
:10347000E15C02E2E16AE552E16EFDEF1FF0060158
:10348000010EC96F120084EC20F0020EE126FE0E40
:10349000DBCFC8F70701C851210A01E1C2D0010AF8
:1034A00001E1A9D0600A01E18AD0010A6BE0530A68
:1034B0005AE0030A4FE0010A44E0160A3CE0030A1E
:1034C00031E0010A28E0070A15E0010A11E0030AC9
:1034D00001E0BBD00A0E94EC20F00701030ECC6F84
:1034E000140ECD6FCE6B09015B6B8CEC0DF0ADD083
:1034F000CC6BABD0E668B1EC20F0E668E66A64EC31
:1035000020F006EC48F0FDEC41F00701020ECC6F14
:1035100009EC20F09AD0050ECC6F0A0E09EC20F0D1
:103520000A0E5FD0060ECC6F020ECD6FCE6BC96B4C
:10353000FDEC41F08AD0E66AA6EC1FF0DAEC41F02F
:1035400084D0090E94EC20F02CEC20F0520EFD6F8C
:10355000930E79D0080E94EC20F02CEC20F05E0E47
:10356000FD6F930E70D0070E94EC20F00701030E50
:10357000CC6F230ECD6FCE6BC96B0601680EFD6F4D
:10358000930E61D0050EE66EB1EC20F00701CA077C
:10359000000ECB5BD880CA55000ECB5506E2070E55
:1035A000F2EC1FF00701400E05D0080EF2EC1FF000
:1035B0000701020ECC6F060ECD6FCE6B46D0050E06
:1035C00094EC20F09DEC20F0BBEC1FF011E080505B
:1035D000010B0EE10701020ECC6F3C0E09EC20F04E
:1035E000020EE7EC1FF00601D70EFD6F680E2BD020
:1035F0000701200EC86F020E94EC20F00601CB6B81
:103600000701CC6BC96B0901590507E0050E595D2F
:1036100004E0780E0701D16F02D00701D16BD26BA5
:1036200014D0060E94EC20F0020EE7EC1FF0070118
:10363000030ECC6FF00ECD6FCE6B90EC0DF006014B
:10364000B50EFD6F930EFE6FC3DE020EE15C02E26B
:10365000E16AE552E16EFDEF1FF0FE0E0701E85D45
:1036600017E10901590505E0050E595D02E006EC78
:1036700020F0E7C7E6FFB5EC20F0D30EE66E070EAC
:10368000E66EB9EC25F0006E050EE15E005012000A
:10369000FF0EE85D07E0B5EC20F004EC12F0E55217
:1036A000E5521200C851200A01E178D1600A01E117
:1036B000D3D0610A01E1ABD0330A01E17FD0030A24
:1036C00052E0010A14E0110A01E01200020EE75D67
:1036D00001E25CD255EC20F001E058D24B0E015DC6
:1036E00001E054D2ADEC20F0100E01EF20F0040EFA
:1036F000E75D23E360EC20F020E1430E015D1DE176
:10370000530E025D1AE14D0E035D17E1B5EC20F09A
:10371000BCEC3FF0E552E552F3CFE9FFF4CFEAFF0E
:10372000E906000EEA5A000EE926070EEA22EF50DB
:10373000310818E0030EA4EF20F00701C95101E0A1
:1037400025D2020EE75D01E221D255EC20F001E026
:103750001DD24B0E015D01E019D2ADEC20F0110E2F
:1037600001EC20F01200080EE75D12E360EC20F09F
:103770000FE1430E015D0CE1500E025D09E1490EBF
:10378000035D06E1520E075D18E0040EA4EF20F081
:103790000701C95101E0FAD1020EE75D01E2F6D15D
:1037A00055EC20F001E0F2D14B0E015D01E0EED1CD
:1037B000ADEC20F0120E01EC20F01200060EE75DD9
:1037C00015E360EC20F012E1490E015D0FE1500EAF
:1037D000025D0CE1520E035D09E1390E065D06E063
:1037E0000601E30EFD6F930E1FEF20F0020E07019E
:1037F000E75D01E2CBD155EC20F001E0C7D14B0EE3
:10380000015D01E0C3D1ADEC20F0210E3DD0020EF0
:10381000E75D0CE355EC20F009E14B0E015D06E19C
:103820000A0E0701CA6FCB6B400E2ED0050E0701A2
:10383000E75D07E3450E0701005D03E1520E015D00
:1038400009E00A0EE66EE66ACC0E006E680E70DBCA
:1038500001E09CD1020E18D0020EE75D17E3450E81
:103860000701005D13E1520E015D10E1020E070138
:10387000C95D03E0030EC95D02E1410E05D0050EEE
:10388000C95D01E08AD0030E01EF20F0020E0701AE
:10389000E75D06E355EC20F003E14B0E015D0BE024
:1038A000530E0701005D03E1480E015D04E0050EC3
:1038B0000701C95D59E10701E76B1E0ECD6FCE6BA5
:1038C00009015A6B020E83DB0701C92BC951080A93
:1038D00049E00F0A3AE0010A33E0030A2CE0010A4A
:1038E00025E0070A1DE0010A0AE0030A01E01200D0
:1038F0000601B80EFD6F680EA2DB050E0CD00601A6
:10390000AB0EFD6F680E9BDB050E97EC20F0060EEC
:1039100097EC20F0070E1DDBB50EFD6F680E20D072
:10392000040EA3DB9D0EFD6F680E1AD006018F0EEC
:10393000FD6F680E15D00601850EFD6F680E10D064
:1039400006016D0EFD6F680E0BD0030E8EDB590E57
:10395000FD6F680E74DB040EFCDA4F0EFD6F680E0F
:103960001FEF20F0200E0CD0070EE75D0BE3080ED2
:10397000E66EE66A460E006E680EDADA03E1020EC3
:1039800001EF20F00B0EE66EE66A3A0E006E680E4E
:10399000CFDA01E0FBD0020E34DB1200050EE66E3A
:1039A000E66A340E006E680EC3DA24E12C0E0701BD
:1039B000085D03E1070E091502D0070E071509017E
:1039C000596FE80403E0050E595D05E10701D16B6D
:1039D000D26BE66A0AD00701D151D21101E0D6D0EC
:1039E000780ED16FD26B010EE66EE66ADFEC47F01F
:1039F000E55255D0050EE66EE66A2E0E006E680E94
:103A000097DA0FE10901590504E0050E595D01E05F
:103A1000FDDA010EDCDA0601C40EFD6F930E1FEF16
:103A200020F00A0EE66EE66A230E006E680E80DA5B
:103A300004E109015A511EE113D0070EE66EE66A51
:103A40001B0E006E680E74DA2CE1110EE66EE66A4B
:103A5000090E006E680E6CDA11E109015A510AE193
:103A6000010EE66EE66E30DB93EC0DF011EC0EF01D
:103A7000A2EC0DF00901010E5A6F120009015A6BF8
:103A8000020EE66E6EDB0901590504E0050E595D74
:103A900001E07CD090EC0DF0400EE66EF4DCE552D7
:103AA0001200050EE66EE66A030E006E680E40DA3E
:103AB00012E12C0E0701085D09E1070E0715006EE3
:103AC000070E06150A0DF350002402D0070E061546
:103AD00009015C6F1200070EE66EE66AFB0E006ECF
:103AE000670E26DA08E00B0EE66EE66AEF0E006E51
:103AF000670E1EDA03E10601CB6B1200090EE66EBB
:103B0000E66AE50E006E670E13DA3CE0060EE66E1E
:103B1000E66ADE0E046E670E056E066A04C0E6FFF6
:103B2000E66E06C0E6FFE5DA076E070EE15E0750B7
:103B3000000928E00A0EE66EE66ACC0E086E680EF2
:103B4000096E0A6A08C0E6FFE66E0AC0E6FFD1DA2F
:103B50000B6E070EE15E0B50000914E00B0EE66ED3
:103B6000E66A3A0E0C6E680E0D6E0E6A0CC0E6FF29
:103B7000E66E0EC0E6FFBDDA0F6E070EE15E0F5077
:103B8000000904E190EC0DF0400E3BDA12002EDA51
:103B900041E0220A3DE0230A2EE0330A23E0030A33
:103BA00019E0010A0FE0110A01E0E7D0050ECD5D32
:103BB000000ECE5902E2020E15DA0601C00EFD6FAC
:103BC000930E17D086DA01E0D8D00601520EFD6FB1
:103BD000930E0FD07EDA01E0D0D006015E0EFD6FAD
:103BE000930E07D076DA01E0C8D00601680EFD6FAB
:103BF000930E25DAC2D0140ECD5D000ECE5901E32E
:103C0000BCD0060EE66EE66ADFEC47F0E55228D03F
:103C1000010E23D0FF0EE85D09E0EA0503E1EA6B3F
:103C2000E86910D0EA51010801E2EA07000ED880E5
:103C3000D155000ED25508E2D107000ED25BD1510A
:103C4000D21102E1210E09D00601CB5100080AE28F
:103C5000CB2BCB513C0806E2400EE66E43EC1AF04B
:103C6000E5528BD00901590504E0050E595D01E0CC
:103C700084D00601FB51FC1109E00601CA0506E1EA
:103C80000601CB5103E1EDEC12F077D00601C851EB
:103C900000081FE20601CA051CE10A0E98D90601B8
:103CA000C80508E1040E0901095D04E0030E0901DD
:103CB0000A5D04E1020E0601C85D03E16FEC15F038
:103CC00005D0030EC85D02E1DEEC15F00601C86BFD
:103CD00054D00501C851000821E20A0E78D9C9D98B
:103CE0000501C80508E1040E0901095D04E0030EA1
:103CF00009010A5D04E1020E0501C85D04E10FDA65
:103D0000F9EC20F006D0030EC85D05E108DABAEC44
:103D100021F0E552E5520501C86B2FD00601C90517
:103D200015E10601CA0512E109015B5100080EE226
:103D30000601CB510BE10601C96B0A0E48D993EC81
:103D40000DF052EC10F092EC0EF015D0090112516A
:103D5000000813E20801D45100080FE20601CB511C
:103D60000CE109015B51000808E2020E30D993EC26
:103D70000DF072EC0FF0A2EC0DF0020EE15C02E22D
:103D8000E16AE552E16E39D10701C851200A01E02C
:103D900012000601CB51000802E242EF20F0EAD9FE
:103DA00012E0020E14D90601C90EFD6F930EFE6FCC
:103DB000E8EC19F008014151000803E2010E07D9AF
:103DC000F9D7020E04D9120011D91CE10601CB511A
:103DD000000802E257D916D009015A050FE109017E
:103DE0005B5100080BE293EC0DF00B0EC4D801E020
:103DF000F3D80C0EC0D801E0EFD812D9010E07019C
:103E0000C919C96F020EE15C02E2E16AE552E16E96
:103E1000F4D01200EBD846E1050E0901135D27E24C
:103E2000800E09010E1523E10701EC5110E1090193
:103E30005A050EE10601CB510BE193EC0DF0EBECD2
:103E400015F0A2EC0DF00701480EEC6F01D0EC0765
:103E50000701EB510AE10DD962D9D2EC21F0E5520C
:103E6000E5520701480EEB6F06D0EB0704D00701BF
:103E7000060EEB6FEC6F09015A0514E109015B5165
:103E800011E10601CB51000802E2FCD80BD093EC03
:103E90000DF00B0E70D801E09FD80C0E6CD801E02D
:103EA0009BD8BED8020EE15C02E2E16AE552E16E07
:103EB000A4D00701CF2B000ED023CC5100080DE277
:103EC000E7D8CD07000ECE5B0050011006E1CCC74D
:103ED000E6FF43EC1AF0E55201D059DEABD81E0ED6
:103EE0002D6E2E6A00D901E14FDF44D901E16CDF6C
:103EF000A1D82C0E2D6E010E2E6EF5D801E189DFB2
:103F000099D8580E2D6E020E2E6EEDD806E182DF86
:103F1000580E0701CF5F020ED05B12001200800E18
:103F2000946E46EC46F00901596B010E01EF20F04A
:103F3000016E026A00C0E6FFE66E02C0E6FFD9D855
:103F4000036E070EE15E0350000912000AD9ADEFBF
:103F500020F0E66E6FEC44F0E552F3CF00F0F4CFC2
:103F600001F0F3CFE6FFF4CFE6FFFAEC19F0E552EB
:103F7000E55206011200E66EBFD8DECFE9FFDDCFC5
:103F8000EAFFEF501200DFEC4AF024C000F025C039
:103F900001F0245025101200EA6A000FE96E070EA6
:103FA000EA221200036E046A02C0E6FFE66E04C055
:103FB000E6FFB5D848EC40F0056E050EE15E055011
:103FC000F3CF00F0F4CF01F0F350F4101200E66EDE
:103FD000EDEC41F0E5521200A2D8FBEC10F0E552F6
:103FE000E5521200E66EE66A64EF20F08DD8020E0C
:103FF000E1260701C851200A1200E552E7CFD9FF98
:104000001200E66E43EC1AF0E552120096D8ADEFBE
:1040100020F0CD6FCE6BC96B09015B6B90EF0DF09B
:1040200092EC0EF072EC0FF08AEC0FF052EC10F004
:10403000A2EF0DF0CFC700F0D0C701F01200FE6F65
:10404000E8EF19F030EC43F0E552E552F3CFE9F731
:1040500007013C0EEA6F12000701030ECC6F5F0EE2
:10406000CD6FCE6BC96B06011200E66E7AD80601E1
:104070001200E66A7CEF20F0E751006E016AC80E7C
:1040800000181200050E0701CF5F000ED05B120072
:10409000CDC700F0CEC701F01200FD0EDBCFE9FF67
:1040A000FE0EDBCFEAFFEF5012004F0E0701005D5E
:1040B0001200FDC6F6FFFEC6F7FF0800F55012001D
:1040C0002B0E0701005D1200DFEC47F0E552E552D0
:1040D0001200DEDF030E2D6E2E6ACDC728F0CEC78C
:1040E00029F0C3EF1FF0CFC728F0D0C729F0C3EFE6
:1040F0001FF03BD8BEEF3EF06FEC44F0E552F3CF3B
:10410000DEFFF4CFDDFF1200D9CFE6FFE1CFD9FF0C
:104110001200E751E72B40DFDFCFEFFF1200DECFC9
:10412000E6FFDDCFE6FF1200E66EA6EF1FF011DF1F
:10413000A70EFD6F680E1FEF20F00701D16BD26B49
:104140000901050E596F12004DDF0701010EC96FFD
:104150001200E75121DFEF6A1200E66AE66A64EFB7
:1041600020F0010EE66E64EF20F0000EE66E070E02
:10417000E66E12005FDF3C0E2D6E2E6A73EF20F0AC
:10418000AFEC26F00601590EFD6F6E0E81EC27F0A4
:104190008FEC26F0DAEC27F00601550EFD6F6E0E5F
:1041A00081EC27F0020E0BEC27F0B4EF26F0AFEC19
:1041B00026F00801DAB50AD065EC27F0F0C8FDF664
:1041C000F1C8FEF6E8EC19F0BEEC26F0B4EF26F0EC
:1041D000AFEC26F00801DAB50AD065EC27F0F2C89A
:1041E000E6FFF3C8E6FFDAEC27F0BEEC26F0B4EF0A
:1041F00026F061EC27F00801DAB5B4D00BEC27F01B
:1042000065EC27F009010EA54AD009010B51040AFB
:1042100015E0070A0EE0020A07E0010A16E10601AE
:10422000470EFD6F6E0E0ED006013C0EFD6F6E0E3A
:1042300009D00601330EFD6F6E0E04D00601240E68
:10424000FD6F6E0EFE6FE8EC19F0090109510F0ABF
:1042500021E0020A1AE0090A13E0060A0CE0030A48
:1042600005E00601C00EFD6F6D0E1DD006011B0E90
:10427000FD6F6E0E18D00601050EFD6F6E0E13D089
:104280000601F70EFD6F6D0E0ED00601E30EFD6FF9
:104290006D0E09D00601D10EFD6F6D0E04D0060122
:1042A000B30EFD6F6D0E81EC27F00601A30EFD6FBE
:1042B0006D0E81EC27F0020EE66EA6EC27F0CFEC37
:1042C00026F04D080DE114C9E6FF15C9E6FF9D0E65
:1042D000006E6D0E49EC27F0070EE15E035031D001
:1042E00014C900F015C901F0040ED890003601364B
:1042F000E804FBE1050E0026000E01220A0E2D6ED9
:104300002E6A00C028F001C029F0DFEC4AF028C076
:1043100000F029C001F028C0E6FF29C0E6FF970E93
:10432000026E6D0E036E046A02C0E6FFE66E04C004
:10433000E6FFDFEC27F004EC49F0056E070EE15EC6
:1043400005505EEC27F006018F0EFD6F6D0E81ECBF
:1043500027F009011351E66EE66A8A0E006E6D0EB3
:1043600096EC27F0020EE15C02E2E16AE552E16EB2
:10437000B4EF26F061EC27F00801DAB50BD00BECB6
:1043800027F0CFEC27F00D0EFD6F750E81EC27F0B6
:10439000BEEC26F0020EE15C02E2E16AE552E16E5B
:1043A000B4EF26F061EC27F00A0E0BEC27F065EC79
:1043B00027F009011351E66EE66A580E006E6D0E85
:1043C00096EC27F0050E0BEC27F0020EE15C02E202
:1043D000E16AE552E16EB4EF26F061EC27F0E66A9F
:1043E0009DEC26F003EC27F08FEC26F010EC27F084
:1043F00002E1010E06D00801DAB302D0F2EC27F098
:10440000000E006E020EE15C02E2E16AE552E16E2E
:104410000050B4EF26F061EC27F0010E93EC27F08A
:1044200003EC27F02EEC27F010EC27F002E1010E50
:1044300006D00801DAB302D0F2EC27F0000E006ECD
:10444000020EE15C02E2E16AE552E16E0050B4EF77
:1044500026F061EC27F0B1EC27F000C0E6FF01C0C8
:10446000E6FF8FEC26F0BCEC3FF0A2EC27F0E7CFA4
:1044700001F0E552E7CF00F00050F3240801EE6FA1
:104480000150F420EF6FEEC800F0016EFD0EDB501E
:10449000001807E1FE0EDB50011803E1F36AF46A2D
:1044A00016D0FD0E3FEC27F0AEEC27F008E0CFEC85
:1044B00026F005E0DF2A010EF7E3DB2AF5D7AEECA4
:1044C00027F003E199EC27F0EF6A28EC27F0020EC1
:1044D000E15C02E2E16AE552E16EB4EF26F061ECE4
:1044E00027F0FD0E3FEC27F0CFEC26F005E0DF2AA9
:1044F000010EFAE3DB2AF8D7DECF00F0DDCF01F0C2
:104500000801EE51001806E1EF51011803E1F36ACA
:10451000F46A21D0DF2A010E01E3DB2AD9CFE9FFBB
:10452000DACFEAFFFD0EEECFDBFFFE0EEDCFDBFFB5
:10453000AEEC27F008E0CFEC26F005E0DF2A010E14
:10454000F7E3DB2AF5D7AEEC27F003E199EC27F08F
:10455000EF6A28EC27F0020EE15C02E2E16AE55224
:10456000E16EB4EF26F0CCEC27F003E04FEC27F03F
:1045700003E153EC27F00AE0E66ADFDB420E006E4F
:104580006D0E49EC27F0070E6CEC27F0020EE15C93
:1045900002E2E16AE552E16EE7D3E1DB4FEC27F09E
:1045A0000CE0BDDBE66AB4EC44F0A2EC27F00801B5
:1045B000D00EF06F730E56EC27F0D6D3CCEC27F06C
:1045C00003E04FEC27F003E153EC27F00BE0010E82
:1045D00093EC27F02E0E006E6D0E49EC27F0070EBF
:1045E0006CEC27F0020EE15C02E2E16AE552E16E5A
:1045F000BBD3C6EC27F009E099DB010EC5DB08014F
:10460000FD0EF06F730E56EC27F0AED38DEC27F055
:1046100003E04FEC27F003E153EC27F028E008011A
:10462000DAB525D0020E0BEC27F0CFEC27F0310ED7
:10463000FD6F750E3CEC27F044C9E6FF45C9E6FF67
:1046400046C9E6FF47C9E6FFD2EC27F006012C0E6B
:10465000FD6F6D0E3CEC27F048C9E6FF49C9E6FF47
:104660004AC9E6FF4BC9E6FFD2EC27F087DB7CD3D3
:104670008DEC27F003E04FEC27F003E153EC27F03B
:1046800004E04DDBB6DDE552E5526ED368DB030E88
:10469000E1265CDB03E04FEC27F003E153EC27F06D
:1046A00033E00801DAB530D0CFEC27F0240EFD6FEF
:1046B0006D0E81EC27F0DF6A200EDF5C24E2DFCF95
:1046C000E6FF6FEC44F0E552DE52F3CFDEFFF4CFAD
:1046D000DDFFDD52010EDBCFE9FF020EDBCFEAFF8B
:1046E000EF500FE0DFCFE6FFE66A1E0E006E6D0EA4
:1046F00010DB010EDBCFE6FF020EDBCFE6FFDAECCC
:1047000027F0DF2AD9D73ADB030EE15C02E2E16A47
:10471000E552E16E29D323DBE652020EDF6EC3DBE6
:1047200018E090EC27F015E0200EDF5C10E2ECDBE7
:104730000EE00CDB2D0804E14BDB02E138DB01D09D
:10474000F5DADF50DF2A20DBF1DAD0DBEDD7C9EC78
:1047500027F0E55209D3CCEC27F002E0A0DB02E120
:10476000A2DB1BE00801DAB518D0CFEC27F0160E5B
:10477000FD6F6D0EC6DB080ED6DB070E006E6D0EEC
:10478000C8DA020ED0DBFC0E006E6C0EC2DA030E2D
:10479000CADBE90E006E6C0EC9DB020EE15C02E2C0
:1047A000E16AE552E16EE0D2F1DB12E0B9DB10E044
:1047B000BDDA080E8DDB07E0B9DA020E89DB03E013
:1047C000B5DA030EE1DAF8EC27F05EEC2EF034DB1C
:1047D000CBD2E2DB02E063DB02E165DB30E0080123
:1047E000DAB52DD0DCDBE30EFD6F6C0E8ADB050E37
:1047F0009ADBDA0E006E6C0E8CDA060E94DBD00EAD
:10480000006E6C0E86DA070EDFDB0601CA5105E08A
:104810000601A10EFD6F6C0E08D0200E0701C85DC9
:1048200006E10601800EFD6F6C0E6BDB07D0C851F0
:10483000E66EE66A5D0E006E6C0E6BDA9FDA020EB3
:10484000E15C02E2E16AE552E16E8ED29FDB1CE0A0
:1048500067DB1AE06BDA050E3BDB15E077DA2D0833
:1048600004E1B6DA02E1A3DA01D060DA060E30DB49
:104870000AE06CDA2D0804E1ABDA02E198DA01D043
:1048800055DA070E81DA85DB6FD286DB02E007DBC3
:1048900002E109DB16E00801DAB513D080DB550E22
:1048A000FD6F6C0E2EDB040E3EDB4D0E006E6C0EAB
:1048B00030DA090E89DB0A0E36DB3F0E006E6C0E15
:1048C00035DB020EE15C02E2E16AE552E16E4CD2B8
:1048D0005DDB0EE025DB0CE029DA040EF9DA07E0F7
:1048E00025DA090EF5DA03E021DA0A0E4DDA51DB9A
:1048F0003BD213DB02E0D3DA02E1D5DA20E0080193
:10490000DAB51DD04CDB390EFD6F6C0EFADA0801FA
:10491000F451E66EE66A2C0E006E6C0EFAD90801B0
:10492000F551E66EE66A1F0E006E6C0EF2D90701B5
:10493000C851E66EE66A0C0E006E6C0EF7DA14D201
:104940000EDAE65203DA02E0AADA02E1ACDA21E09A
:104950000801DAB51ED023DB020EFD6F6C0ED1DA32
:10496000DF6A100EDF5C14E280DAEF500FE07DDAD0
:10497000EF50E66EE66ADFCFE6FFE66AFA0E006EFB
:104980006B0E87DA090EE15E035098DADF2AE9D769
:10499000F5D9E552E9D1E3D9E65285DA26E0C0DA65
:1049A00024E0C4D94FDADF6EC1D9A0DA000EDF5C93
:1049B0001CE3100EDF5C19E2A7DA17E0BFDA55DA64
:1049C000E552E750EF6E080EDF5C05E3AFD9080E45
:1049D000DF5C180FD9D90F0EDF5C02E15EEC2EF020
:1049E0000801390EF06F740E61DAE552BDD1CEDAEE
:1049F00009E0A4DA09EC33F0E55208014F0EF06F3C
:104A0000740E54DAB1D1C2DA08E090D9020EE66E23
:104A1000F5D9620EF06F740E49DAA6D1B7DA08E064
:104A200085D9030EE66EEAD9790EF06F740E3EDA80
:104A30009BD1ACDA07E07AD9E66AE0D9920EF06F42
:104A4000740E34DA91D1A2DA08E070D9010EE66E64
:104A5000D5D9A70EF06F740E29DA86D197DA3EE029
:104A60005FDA3CE063D96BEC40F0E552E552030EAF
:104A7000E66EE66AF60E006E6B0E1CDA02E1E66A7E
:104A80001ED0030EE66EE66AF20E006E6B0E12DAB0
:104A900002E1010E13D0030EE66EE66AEE0E006E22
:104AA0006B0E08DA02E1030E09D0030EE66EE66A29
:104AB000EA0E006E6B0EFED911E1040EE66E53ECA9
:104AC00032F0E55233D93FD904E038DA5DEC32F008
:104AD000E5520801C30EF06F740EE8D945D11DDA16
:104AE00002E0DDD902E1DFD90AE0010EE66E67ECF3
:104AF00032F0E5520801E00EF06F740ED7D934D1D0
:104B00000CDA02E0CCD902E1CED909E0E66A67EC22
:104B100032F0E5520801F70EF06F740EC7D924D1B8
:104B2000FCD902E0BCD902E1BED910E00901025172
:104B3000E66EE66A0151E66EE66A0051E66EE66AE6
:104B4000CA0E006E6B0EA5D90B0EC6D90DD124DA94
:104B500002E0A5D902E1A7D905E0030EE66E43EC19
:104B60001AF0E552020EE15C02E2E16AE552E16E02
:104B7000FBD0F5D8040EE126FB0E81D910D917E041
:104B8000EDD915E00CD960080DE2D3D9EFCF00F0D4
:104B90007B0E005C07E203D9E00FE66ECAD9E5524E
:104BA000E750EF6EDF2A010EE9E3DB2AE7D7D6D91B
:104BB00004E1DF2A010E01E3DB2A020EDB6A030EA9
:104BC000DB6A020EDBCFF6FF030EDBCFF7FF1B0E17
:104BD000F702F3CFF7FFF602F3CFF6FFF450F72614
:104BE000B70EF626750EF7220800F55001E184D0C5
:104BF000020EDBCF02F0030EDBCF03F01B0E03022D
:104C0000F3CF03F00202F3CF02F0F4500326B70E05
:104C10000226750E0322046A02C0E6FF03C0E6FF07
:104C200004C0E6FFCAEC3FF08DD927C000F028C0D1
:104C300001F027C0E6FF28C0E6FF020EDBCF05F03B
:104C4000030EDBCF06F01B0E0602F3CF06F00502C3
:104C5000F3CF05F0F4500626B70E0526750E062292
:104C6000076A05C0E6FF06C0E6FF07C0E6FFF6D804
:104C7000BEEC3EF0086E070EE15E0850000935E11B
:104C8000020EDBCFE9FF030EDBCFEAFFD890E93657
:104C9000EA36C90EE926050EEA22EECF00F0EFCF84
:104CA00001F0DECFE6FFDDCFE6FFFB0EDBCFE6FF58
:104CB000FC0EDBCFE6FFFA0EDBCFE6FFFB0EDBCF11
:104CC000E6FFFC0EDBCFE6FFFD0EDBCFE6FFFE0EC0
:104CD000DBCFE6FF04D001C0FAFF0050F96EFBDF26
:104CE000026E090EE15E02500DD0020EDB2A030EA9
:104CF00001E267D7DB2A65D7B1D811D849EC15F0A6
:104D000021D9E552040EE15C02E2E16AE552E16E6E
:104D10002BD0BFD8070EE15E03505EEF27F0FD0EEB
:104D2000DBCFE6FFFE0EDBCFE6FF1200F60EDBCF99
:104D3000E6FFF70EDBCFE6FF120008D9DECFE6FF75
:104D4000DDCFE6FF1200D2D884EF27F011D9EF5063
:104D50001200EDEC21F0E552E55200091200D9CF26
:104D6000E6FFE1CFD9FF1200E552E7CFD9FF1200ED
:104D70000BEC22F0E7D8E552000912000601530EB1
:104D8000FD6F6E0E81EF27F0E66EB4EC44F0A2EFFB
:104D900027F029EC22F0F3D8F350F4101200C9D810
:104DA000EF501200D7EC20F0E552E5521200010E50
:104DB000E76EF60EDBCF00F0F70EDBCF01F0E75029
:104DC0000026000E012200C0E6FF01C0E6FF12002F
:104DD000010EE76ECDD8E750E926000EEA22EF502B
:104DE0001200C0EC20F0E552E5521200BEEC3EF09D
:104DF000036E070EE15E03500009120071EC32F001
:104E0000A1D808011200BCEC3FF0B9D8F3CFE6FFFF
:104E1000F4CFE6FF1200E66EEDEC41F0E552120031
:104E2000DECFE6FFDDCFE6FFEFEC3FF0026E060ED1
:104E3000E15E025000091200400EE66E43EC1AF0EB
:104E4000E552120030EC43F0E552E552F350120007
:104E500088D800C0F3FF01C0F4FF1200FB0EDBCFC7
:104E6000E6FFFC0EDBCFE6FF1200DF50EA6ACC0F54
:104E7000E96E080EEA22120044D8DFEF27F0DBCFFC
:104E8000DEFFDBCFDDFF1200E8EC20F0E552E5525B
:104E90001200A0D894D804EC49F0036E120046DF4B
:104EA0003EDFB8EF26F03BDFA9EF26F0F16F37DFEA
:104EB000D2EF26F08FD83ADFF6EF26F080D8DAEF7F
:104EC00027F04DDF020EE126120029DFF1EF26F078
:104ED0005BDF2CDFA3EF26F0E15E03500801000E3C
:104EE000F26F060EF36F1BDF44EF27F06FEC22F03A
:104EF000E552E552F60EF3CFDBFFF70EF4CFDBFF02
:104F00001200FE6FE8EF19F0D950F60FE96EFF0EB0
:104F1000DA20EA6EEE50ED10120021DFA6EF26F047
:104F200005DFC9EF26F0E66E9DEF26F0F2DEBEEF5C
:104F300026F0DECFE9FFDDCFEAFF1200F7DE82DFE9
:104F4000E66E1200E552E552E55212006FEC44F0B5
:104F5000E552F3CFDEFFF4CFDDFF120020DF2008A3
:104F60001200FD0EDBCF00F0FE0EDBCF01F01200D1
:104F7000F60EDBCFE9FFF70EDBCFEAFF1200E552BA
:104F8000E552F3CF00F0F4CF01F01200E8DE53EF6A
:104F900027F02ED81CEF27F094DFA6EF26F095DF40
:104FA000060112000BEC42F0006E060EE15E0050AE
:104FB0005EEF27F0FAEC19F0E552E5521200000E10
:104FC000E66E060EE66E1200AEDFC20E006E6C0ECE
:104FD00089EF26F0016E026A00C0E6FFE66E02C0AD
:104FE000E6FF12000801BE0EF06F730E56EF27F0B9
:0C4FF00008011F0EF06F740E56EF27F042
:044FFC003AEC2DF06E
:10500000FB0EDBCFF3FFDB06F35000090AE088EC70
:105010002DF0FA0EF3EC2DF0F3E1011CF1E1010E9D
:1050200001D0000E69EF2DF03AEC2DF03B0EE1249B
:1050300002E3E168E652E16E010EDB6A020EDB6A12
:10504000F90EDBCFF6FFFA0EDBCFF7FFFB0EDBCF5F
:10505000F8FF0800F550DF6EDF5002E18DEF2CF015
:10506000250EDF5C02E080EF2CF0030EDB6A040EFD
:10507000DB6A050EDB6A060EDB6A070EDB6AA2EC52
:105080002CF02D0EDF5C0CE02B0EDF5C09E0200E17
:10509000DF5C06E0230EDF5C03E0300EDF5C1AE12C
:1050A000DF50300A14E0130A0FE0030A0AE00B0A8B
:1050B00005E0060AE4E1030EDB80E1D7030EDB82A4
:1050C000DED7030EDB84DBD7030EDB86D8D7030ED7
:1050D000DB88D5D72A0EDF5C1BE19EEC2CF0ECECD4
:1050E0002CF010E0030EDB8028682968130EDBCF5C
:1050F0002DF0140EDBCF2EF091EC3EF0040E26C006
:10510000DBFF03D0130ED5EC2CF0A2EC2CF00BD06F
:10511000090EDB6A43EC2DF003E0B7EC2DF0FAD773
:10512000090ED5EC2CF0030EDBB0DB982E0EDF5C05
:105130001BE1A2EC2CF02A0EDF5C0BE19EEC2CF0C4
:10514000ECEC2CF003E1130E27EC2DF0A2EC2CF08C
:105150000BD0090EDB6A43EC2DF003E0B7EC2DF029
:10516000FAD7090E27EC2DF0680EDF5C07E1A2EC00
:105170002CF0680EDF5C1DE1030E18D0740EDF5CAE
:1051800017E07A0EDF5C14E0480EDF5C06E0540E98
:10519000DF5C03E05A0EDF5C02E1020E07D06C0E0A
:1051A000DF5C03E06A0EDF5C04E1010E7AEC2DF0B7
:1051B000C9DBDF506E0A01E17FD31E0A01E192D103
:1051C000200A01E18FD13F0A01E149D11A0A01E128
:1051D00046D10D0A01E143D1200A01E140D13A0A4A
:1051E00001E13DD1200A01E13AD1260A01E135D1A0
:1051F0000D0A01E132D11A0A01E1D9D0200A4AE0B0
:10520000300A1FE0460A0EE0250A01E083D3D95098
:10521000F90FE96EFF0EDA20EA6E010EEE5E000E67
:10522000EE5AEE5A88EC2DF0250EE66E95DB03E182
:10523000011C01E169D384EC2DF001E26BD3DB2A80
:1052400069D3080EDB6A040EDB50010806E2040E87
:10525000DB044CEC2DF0DB508BDB080EDB5009E05F
:10526000030EDB50010B05E172DB01E04DD3080EAC
:10527000DB6A64DBEFCFDFFFFCEC2DF003E1011C08
:1052800001E142D384EC2DF001E3DB2A60DB01E194
:1052900041D33AD3070EDB5002080FE1C8EC2DF0E2
:1052A000030E8FEC2DF00E0EEECFDBFF0F0EEECFC8
:1052B000DBFF100EEECFDBFF20D0F70EDBCF03F0CD
:1052C000F80EDBCF04F0020E035E000E045AF70E58
:1052D00003C0DBFFF80E04C0DBFF03C0E9FF04C01E
:1052E000EAFF7FEC2DF0026A0E0E00C0DBFF0F0E0E
:1052F00001C0DBFF100E02C0DBFF0E0EDBCFE6FFAE
:105300000F0EDBCFE6FF100EDBCFE6FFCAEC3FF05F
:10531000E552E552E552130E27C0DBFF140E28C0FC
:10532000DBFF060EDB5005E0130EC3EC2DF001E2AF
:105330006ADBE7EC2DF002E2130E37DBAAEC2DF06E
:1053400006E0040EC3EC2DF002E2050E2EDB030E88
:10535000DBB005D0FCDA01E0D7D2080EDB6A090E1B
:10536000DB6A0E0EDBCFF6FF0F0EDBCFF7FF100E62
:10537000DBCFF8FF0800F550DF6EDF5014E0EDECF6
:105380002DF011E2FCEC2DF003E1011C01E1BCD297
:10539000BBDB01E3DB2A090EDB2AD9500E0FE96ED5
:1053A000000ECBDBE7D7D3DA01E1B4D2ADD2C6DA57
:1053B000110EEECFDBFF120EEDCFDBFF110EDBCFB8
:1053C000E6FF120EDBCFE6FFBCEC3FF0E552E55204
:1053D000130EF3CFDBFF140EF4CFDBFF060EDB5012
:1053E00004E0130ED0DB01E20EDBE7EC2DF002E26D
:1053F000130EDBDAAFDB05E0040EC5DB02E2050EBF
:10540000D4DA030EDBB005D0A2DA01E07DD2080EBB
:10541000DB6A090EDB6A110EDBCFE9FF120EDBCF70
:10542000EAFFEFCFDFFFDF5014E0D7DB12E2E4DB6F
:1054300003E1011C01E168D267DB01E3DB2A090E0D
:10544000DB2A110EDB2ADBCFE9FF120EE8E3DB2AB1
:10545000E6D77DDA01E15ED257D2030EDB8E070E6E
:10546000DB0410E195DB040E5ADB0A0EEECFDBFF06
:105470000B0EEECFDBFF0C0EEECFDBFF0D0EEECFF3
:10548000DBFF6CD0070EDB5003082CE1030EDBAE14
:105490000DD0B2DA020E76DAEFCF00F0016A026ABE
:1054A000036A00AE39D00168026835D0F70EDBCF51
:1054B00001F0F80EDBCF02F0020E015E000E025A80
:1054C000F70E01C0DBFFF80E02C0DBFF01C0E9FFF1
:1054D00002C0EAFFEFCF00F00A0E00C0DBFF0B0EA8
:1054E000DB6A38D0070EDB50020809E1030EDBAEA1
:1054F00004D059DB02AE10D00ED055DB0DD0030E18
:10550000DBAE12D079DA020E3DDAF9DA026A036A0A
:1055100001AE02D002680368E2DA0C0E02C0DBFFC3
:105520000D0E03C0DBFF1AD0F70EDBCF02F0F80E32
:10553000DBCF03F0020E025E000E035AF70E02C02C
:10554000DBFFF80E03C0DBFF02C0E9FF03C0EAFF88
:10555000D6DAC5DA0C0EDB6A0D0EDB6A060EDB50FE
:1055600005E1010EF36E050EF3CFDBFF150EDB6ACE
:10557000160EDB6AD950370F006E000EDA20016E6E
:10558000390E00C0DBFF3A0E01C0DBFF380EDB6ACC
:10559000080EDB6A0A0EAEDADF50780A12E0200A43
:1055A00010E0280A0CE0200A0AE03F0A06E00D0A93
:1055B00002E0200A08E1020E05D0080E03D0080E12
:1055C000DF26100E97DA030EDBBE02D0DB92DB94EF
:1055D000DB50800B24E08ADAD890030EEB50000AEF
:1055E00008E6000EEE5C000EEE58000EEE58000EBF
:1055F000EE5815E213DA2B682C682D682E6883ECC0
:105600004AF00A0E22C0DBFF0B0E23C0DBFF0C0E9C
:1056100024C0DBFF0D0E25C0DBFF2D0E08D0030ECE
:10562000DBA202D02B0E03D0DBA408D0200EF36E39
:10563000170EF3CFDBFF150EDB2A02D0170EDB6A45
:10564000050EDB5003E1B7D901E189D0A20E006E4F
:10565000960E016E000E026E070EDBCF03F0046A99
:10566000056A066A03C02BF004C02CF005C02DF0BB
:1056700006C02EF0D3D9BBEC4AF000502224F36EC2
:1056800001502320F46E02502420F86EF4CFF7FF6F
:10569000F3CFF6FF0800090EF5CFDBFF580EDF5CF5
:1056A0000FE1610EF36E090E7BD90AE3200E006E46
:1056B000090EDBCFE7FF0050E75E090EE7CFDBFF07
:1056C000070EDBCF00F0016A026A036A0FDA00C03E
:1056D0002BF001C02CF002C02DF003C02EF0EECF55
:1056E00026F0EECF27F0EECF28F0EFCF29F0BBEC7D
:1056F0004AF029C0EDFF28C0EDFF27C0EDFF26C00E
:10570000EFFF390EDBCFE9FFDB063A0EDBCFEAFF16
:1057100001E2DB06090EDBCFEFFF150EDB2A4BD9CA
:1057200095E1030EDBA61DD06F0EDF5C06E1C1D94B
:1057300018E3150EDB285BDA14D0780EDF5C09E085
:10574000580EDF5C06E0620EDF5C03E0420EDF5CB9
:1057500008E1020EF36E160EF3CFDBFF02D0150E3A
:10576000DB6A030EDB50100B0EE0040EDBCF00F003
:10577000050EDB50D880005406E2060EDB5003E134
:10578000040EDB5034DA95D90AE2050EDBCFE7FFD1
:10579000150EDB50E75E050EE7CFDBFF02D0050EEE
:1057A000DB6A040EDBCF00F0160E45D9D88000541A
:1057B00014E2160EDBCFE6FF150EDBCFE6FF040E7C
:1057C000DBCFE6FF050EDB50E552E75CE552D88003
:1057D000E754E552D880E7545FD9030EDB50010B44
:1057E0000BE1080EDB5008E0B2D801E08DD0080EC6
:1057F000DB50BED8080EDB6A170EDB5007E088D9F5
:10580000170EF1D903E1011C01E17ED0160EDB5029
:1058100016E07ED9300EE66E9FD802E1011C74E0DE
:1058200077D9DFCFE6FF41EC4AF0E552E552E55289
:10583000F4CF01F00001F31C02E1011C65E0050E4C
:10584000DBCF00F0160EDB50D880005409E2050EC5
:10585000DBCFE7FF160EDB50E75E050EE7CFDBFF81
:10586000300EE66E050ECBD94FE1390EDB2ADBCFC9
:10587000E9FF3A0E01E3DB2ADBCFEAFF090EEFCFA7
:10588000DBFFDB500EE044D9090EADD902E1011C6B
:105890003BE0390EDB2ADBCFE9FF3A0EEDE3DB2AF2
:1058A000EBD755D831E1160EDBCFE6FF080EC3D893
:1058B000E552E7245DD82ED0070EDB50030A1CE02A
:1058C000010A14E0030A07E07BD9DBCFEEFF020EEA
:1058D000DBCFEDFF1FD0F5D8056A03AE02D0046818
:1058E00005682CD8BCD805C0EEFF14D0EAD803BE9A
:1058F000046824D8B4D80ED063D9DBCFEFFF0AD028
:105900007BD905E1011C03E1F368F46810D0FCD8F1
:1059100001E3DB2A79D929EF28F0010EDBCF00F073
:10592000020EDBCF01F000C0F3FF01C0F4FF3B0E1D
:10593000E15C02E2E16AE552E16ECBD029D9020EC8
:105940008FEF2DF061D90800F550DF6E1200200EA8
:10595000E66E080EFFEF2DF041EC4AF0E552E552FD
:10596000E552F3CF00F0F4CF01F00001F31C120078
:10597000006E016AD950010F4DD90050EE2601503A
:10598000ED221200045E000E055AF70E04C0DBFF84
:10599000F80E05C0DBFF04C0E9FF05C0EAFF1200F6
:1059A000DBCFF4FFF350F45C1200DB50E76E040E23
:1059B000E7CFDBFF12000A0EDBCF00F00B0EDBCFD0
:1059C00001F00C0EDBCF02F00D0EDBCF03F0005028
:1059D0000110021003101200130EEECFDBFF140EA5
:1059E000EDCFDBFF130EDBCF00F0140EDBCF01F0A9
:1059F0000001800E01141200F70EDBCF04F0F80E48
:105A0000DBCF05F01200050EDB50E66ED950130F08
:105A100001D9E552E750EE6EED6A12000A0EDBCFB7
:105A200026F00B0EDBCF27F00C0EDBCF28F00D0E8F
:105A3000DBCF29F01200DBCFE6FF150EDBCFE6FF50
:105A4000050EDB50E552E724E552E7241200DB5057
:105A5000CED8010EF36E060EF3CFDBFF1200EE5030
:105A6000EFCFEAFFE96E02C0EEFF03C0EEFF04C015
:105A7000EEFF1200D9CFE6FFDACFE6FFE1CFD9FF84
:105A8000E2CFDAFF1200DFCFE6FFE66AF5EC4AF07C
:105A9000E552E552F3501200E76E080EE7CFDBFF48
:105AA0001200EECF00F0EECF01F0EFCF02F0036A6C
:105AB0001200050EDBCF00F0150EDB50D88000542D
:105AC0001200010EDBCF02F0020EDBCF03F0046AFE
:105AD0001200E552E5CFDAFFE7CFD9FF12000A0E38
:105AE00000C0DBFF0B0E01C0DBFF1200D9500A0F14
:105AF0000AEF2EF0F36E070EF3CFDBFF1200EECFAE
:105B000000F0EFCF01F01200010EDB2A020E1200AE
:105B1000FC0EDBCFE6FFFD0EDBCFE6FF1200005EE2
:105B2000000E015AF70E00C0DBFFF80E01C0DBFFCC
:105B300000C0E9FF01C0EAFF1200DA20EA6EEF2A96
:105B4000EECFF6FF000EEF22EECFF7FFEF22EECF03
:105B5000F8FF1200040EDBCFE6FF130EDB50E55218
:105B6000E75C9ADFDB5004DF060EDB501200090E03
:105B7000DB500A0DF350DF24D00FE76E090EE7CF9C
:105B8000DBFFA2EF2CF0DB50F36E050ED0EF2CF014
:105B9000F70EDBCF00F0F80EDBCF01F01200DFCF05
:105BA000E6FFACEF2CF028DF030EECDE51EF2DF01A
:105BB000FEEC27F0E552E552E552E55200091200ED
:105BC000BDDEEE50EFCFEAFFE96E010E1200130EBC
:105BD000DB50F36E040ED0EF2CF0040EDB50F36EAE
:105BE000090ED0EF2CF0DBCFE6FFACEF2CF0E76E28
:105BF000050EE7CFDBFF12008BDFCFEF2DF0DBCF01
:105C0000E6FF86DFD8EF2DF0D950F90FE96EFF0ED1
:0E5C10009DEF2DF0E96E000EDA20EA6E120014
:025C1E00DACFDB
:105C2000E4FFE2CFDAFFE9CFE4FFEACFE4FFF6CF0B
:105C3000E4FFF7CFE4FFF5CFE4FFF3CFE4FFF4CFC9
:105C4000E4FFFACFE4FF00EE20F0140EE80403E3D3
:105C5000EECFE4FFFBD700EE00F0200EE80403E3F4
:105C6000EECFE4FFFBD7E65260BE7BD80F0150BFFA
:105C70009ADAA46AE55200EE1FF0200EE80403E36E
:105C8000E5CFEDFFFBD700EE33F0140EE80403E39D
:105C9000E5CFEDFFFBD7E5CFFAFFE5CFF4FFE5CF8A
:105CA000F3FFE5CFF5FFE5CFF7FFE5CFF6FFE5CF53
:105CB000EAFFE5CFE9FFE5CFDAFF110085EC33F02D
:105CC000020EE1260801540EC76F520EC86FC96B51
:105CD000CA6BCB6B900E6F6E6EAEFED7606A0F0113
:105CE000A00E196F1869016B200E006F506BE00E4B
:105CF0001D6F1C69800E096F680E086F400E0D6FD6
:105D0000800E0C6F116B106F706AD20E716E020EE6
:105D1000726E200E736E0801DB51000802E26F6A9A
:105D200002D0600E6F6ED08EA382A380030EA56E8C
:105D3000020EE66E6FEC44F0E552F3CFDEFFF4CFD7
:105D4000DDFFDECFE9FFDDCFEAFFEFCFFCF8070193
:105D5000F66BFE6B020EE15C02E2E16AE552BBEF1C
:105D600033F00F0E65140701ED6F66CFEEF767CFC6
:105D7000EFF768CFF0F769CFF1F76ACFF2F76BCFA3
:105D8000F3F76CCFF4F76DCFF5F7609EEE51A60AEE
:105D900001E102D2030A01E1D9D1010A01E1CED128
:105DA000070A01E1C1D1350A01E169D1030A01E124
:105DB0002AD11C0A01E1EED0010A01E1DCD00D0A72
:105DC00001E1A8D0010A01E187D0070A67E0010AD2
:105DD0005FE0030A3DE0010A23E08E0A18E0080AAA
:105DE00001E012001B0EEF5D03E1F2C750F90BD08A
:105DF0001A0EEF5D01E0D6D1F251000EF350F325FB
:105E00000901516F526B0901010E586F1200EF51D9
:105E10000901115D02E03FEC1AF0EFC711F9120021
:105E2000EFC713F9F1C701F0006AF051090100242E
:105E3000146F000E0120156FF5C701F0006A07010D
:105E4000F45109010024166F000E0120176F120093
:105E50005CEC33F003E08AEC33F0FDE125EC33F049
:105E600003E091EC33F0FDE12EEC33F003E098EC2D
:105E700033F0FDE100500C240901186F01500D2092
:105E8000196F02500E201A6F03500F201B6F120063
:105E9000EFC720F90901780E546F12005CEC33F063
:105EA00003E08AEC33F0FDE1D0DB03E091EC33F06A
:105EB000FDE1D4DB03E098EC33F0FDE100500C246D
:105EC0000901446F01500D20456F02500E20466FAE
:105ED00003500F20476F12005CEC33F003E08AECB4
:105EE00033F0FDE1B2DB03E091EC33F0FDE1B6DB32
:105EF00003E098EC33F0FDE100500C240901486FF9
:105F000001500D20496F02500E204A6F03500F20A0
:105F10004B6F1200EFC753F90901535129E0F1C744
:105F200001F0006A0701F051090100244C6F000ED6
:105F300001204D6F680E4C1905E1010E4D1902E16B
:105F40004C6B4D6BF00E0701F31504E009014E6B2D
:105F50004F6B0AD0F3C701F0006AF2510901002427
:105F60004E6F000E01204F6F0901780E566F120020
:105F70000901566B1200EFC705F9F4C706F9F1C71E
:105F800001F0006AF05109010024076F000E0120A2
:105F9000086F12004D0E0801FC5D03E1EFC712F916
:105FA00026D0EFC726F0276A286A296A490E2B6E89
:105FB000060E2C6E2D6A2E6A83EC4AF022C026F063
:105FC00023C027F024C028F025C029F0F40E26268F
:105FD000010E2722000E28222922E80E2B6E030E26
:105FE0002C6E2D6A2E6ABBEC4AF026C012F9F1C75E
:105FF00001F0006A0701F05109010024036F000E4F
:106000000120046F1200150E0901095D09E2150E49
:106010000701EF5D05E3030EF05D02E0010EADDB6D
:106020000F0E0901095D09E10D0E0701EF5D05E1A4
:10603000030EF05D02E0010EA0DB0901095107012A
:10604000EF5D05E109010A510701F05D02E03FEC57
:106050001AF0EFC709F9F0C70AF90801DAA104D06C
:106060000F0E0701F21504D00701F3390F0B0F0BC8
:1060700009010B6FF1C70CF9F5C70DF912000F0EEE
:106080000901095D02E10701EF890701EF510901EB
:106090000E5D0AE10701F05109010F5D05E10701FD
:1060A000F1510901105D02E03FEC1AF0400E0901C8
:1060B0000F1509E1400E0701F01505E0100EF0156F
:1060C00002E0030E5ADBEFC70EF9F0C70FF9F1C774
:1060D00010F96BDB1BE109011C511D111E111F1171
:1060E00015E10901185119111A111B110FE018C9F6
:1060F0001CF919C91DF91AC91EF91BC91FF9090193
:106100001C07000E1D5B1E5B1F5B0CD04EDB4AE0C4
:1061100009011C511D111E111F1144E01C6B1D6B48
:106120001E6B1F6B3FEF1AF0EFC733F9F0C734F95E
:10613000F4C735F90901780E556F1200FF6B070E91
:10614000FF5D30E206DBFF51FADAF9D7FF6B070E8D
:10615000FF5D05E2FEDA070EFF25F1DAF8D7410E02
:10616000F15D03E0420EF15D03E10801320E02D061
:106170000801310EC96F380E0701F15D02E1080117
:10618000DA81330E0701EF5D03E10801530E02D0FF
:1061900008014E0ECA6F1200EFC72FF9F0C730F991
:1061A000F1C731F91200B1DAE6520F0E0F015515A1
:1061B0000701ED6F56CFEEF757CFEFF758CFF0F757
:1061C00059CFF1F75ACFF2F75BCFF3F75CCFF4F783
:1061D0005DCFF5F750CFDFFF0F01509F070EDF14A3
:1061E000040830E1020E0701EE5D01E086D00801EF
:1061F000CC51000801E381D0D8DA01E17ED007015B
:10620000F0510901125D01E178D00801DB5100086D
:1062100074E2EEC7F6F7EFC7F7F712C9F8F7F00E1A
:106220000701F115F96FF2C7FAF7F3C7FBF7F4C7E7
:10623000FCF7F5C7FDF70F0140B7FDD725DACCC84D
:10624000FEF75BD0070EDF14020821E10701F151D0
:10625000000804E2F0C73AF9F1C736F9F551000831
:1062600004E2F4C73BF9F5C737F9EF51000804E23F
:10627000EEC73CF9EFC738F9F351000804E2F2C762
:106280003DF9F3C739F90901780E576F36D0070188
:10629000EE51FA0A32E1F1C700F0016A026A036ABC
:1062A000F2C704F0056A066A076A080E1F0B02E0CF
:1062B00031DAFEE17EDAF3C708F0096A0A6A0B6A8E
:1062C000100E1F0B02E02DDAFEE100500824090138
:1062D000406F01500920416F02500A20426F035065
:1062E0000B20436FF5C701F0006A0701F451090163
:1062F00000243E6F000E01203F6FE55267D2000E72
:106300000901E76E5419E8AE02D0543503D0E750C6
:10631000D880545501E25407000E0901E76E551963
:10632000E8AE02D0553503D0E750D880555501E28C
:106330005507000E0901E76E5619E8AE02D0563532
:1063400003D0E750D880565501E25607000E0901E8
:10635000E76E5719E8AE02D0573503D0E750D88022
:10636000575501E257071200D0D9020EE126080165
:10637000D551DE6EDD6A0801F95112E1F3D9015001
:106380000318E8AE02D0033404D00250005C03507E
:10639000015806E2020EF1D90801010EF96F15D07D
:1063A0000801F90512E1DED9020E0226000E0322D1
:1063B00003500118E8AE02D0013404D00050025C52
:1063C0000150035802E20801F96B020EE15C02E29F
:1063D000E16AE552D0D1120012000801FA2B000E3A
:1063E000FB238DDFDDD93C0E2D6E2E6A72D901E1C3
:1063F000BBDFD6D92C0E2D6E010E2E6E6AD901E1AF
:10640000EADFCED9580E2D6E020E2E6E62D906E14D
:10641000E3DF580E0801FA5F020EFB5B1200070172
:10642000FE5102E1CCC8FEF712000701FE5101E166
:106430001200020EF65D13E10801CC5100080FE2D4
:10644000B4D90DE00801DB51000809E2010EE66E47
:1064500007EC4BF0E5520F0140B7FDD715D9070106
:10646000FE0712000F0140B7FDD708D90A0E466F8C
:10647000010E456F080E406F40B7FED712000F01A6
:1064800040B7FDD7FBD8060E466F2C0E476F010EA6
:10649000486F496B4A6B090E4B6F100E4C6F9AD9BF
:1064A00040B7FED7120031D90F0140B7FDD78AD9C6
:1064B000190EC1D840B7FED726D127D90F0140B752
:1064C000FDD780D9020EB7D840B7FED71CD11DD951
:1064D0000F0140B7FDD776D9030EADD840B7FED730
:1064E00012D113D9040EE1264DD9A5EC43F0E552A3
:1064F000E55226C0DEFF27C0DEFF28C0DEFF29C030
:10650000DDFFDD52DD52FE0EDB50020802E14DD907
:1065100053E10F0140B7FDD7B1D80B0E466FFE0E09
:10652000DBCF47FF486B496BE1D800504A6FDED89C
:10653000080E2FD9FEE100500F014B6FD7D8100E77
:1065400028D9FEE100500F014C6F1CD9BCEC3FF084
:10655000E552E552F3CF00F0F4CF01F0040ED890ED
:1065600000360136E804FBE1026A036A180E086E81
:10657000D9CFE9FFDACFEAFFE8501F0BEECF04F0E6
:10658000EECF05F0EECF06F0EECF07F007E0D890A3
:106590000732063205320432E806F9E10F0E04161E
:1065A000056A066A076A05D900C04DFF0F01080E8B
:1065B000456F406F40B7FED7040EE15C02E2E16A2E
:1065C000E552D9D0A2D80F0140B7FDD7FBD81B0E9A
:1065D00032D840B7FED7FE0EDB041AE1F3D81A0E0C
:1065E000476F486B496BFD0EDBCF01F001C000F037
:1065F00001504A6FFF0EE76EFC0EDBCF00F0E75054
:106600000016016A00C04BFF4C6BE4D840B7FED7C0
:106610007AD07BD80F0140B7FDD730D8090E466F2E
:10662000476BFE0EDBCF48FF030E456F080E406F31
:1066300040B7FED768D0476F486B496BFE0EDBCF83
:106640004AFF4B6B4C6BEAEF33F0B3D8F4C708F05A
:10665000096A0A6A0B6A100E1F0B12000850002606
:10666000095001220A5002220B500322F5C70CF0F8
:106670000D6A0E6A0F6A180E1F0B1200406B400E57
:10668000426F200E416F1200406B426B800E416FD3
:10669000F6C746FFF7C747FFF8C748FFF9C749FFE6
:1066A000FAC74AFFFBC74BFFFCC74CFFFDC74DFFB6
:1066B000080E456F406F1200F2C700F0016A026ACF
:1066C000036AF3C704F0056A066A076A080E1F0B1F
:1066D0001200FAC828F0FBC829F0DFEC4AF024C009
:1066E00000F025C001F0245025101200D9CFE9FF99
:1066F000DACFEAFFEECF00F0EECF01F0EECF02F0FE
:10670000EFCF03F01200AEDE61D0D9CFE6FFE1CFCC
:10671000D9FF1200D8900436053606360736E8064B
:106720001200D890083609360A360B36E8061200F1
:10673000D8900C360D360E360F36E8061200EA6A8F
:10674000210FE96E090EEA22E552E750EF6EFF2BAA
:106750001200FF29EA6AEE0FE96E070EEA22EF50F7
:10676000E66E120009011351006E016ADECF02F0DD
:10677000DDCF03F01200E16E29D0E66E1DEC1AF0B9
:10678000E5521200FC0EDBCFE6FFFD0EDBCFE6FF8D
:106790001200D8900332023201320032E8061200B1
:1067A000FAC800F0FBC801F01200800E09010E15B6
:1067B0001200045000260550012206500222075004
:1067C000032212005BDF050E466F1200E552E7CF91
:0E67D000D9FF12004D6B080E456F406F12008E
:0267DE00434C2A
:1067E0004F5345440053454E44204641494C0044D4
:1067F000415441204143434550540053454E4420A9
:106800004F4B002B4353513A0053544154453A20C7
:10681000434F4E4E454354204F4B00535441544533
:106820003A2000434F4E4E454354204F4B002B43DC
:106830004C4950002B43524547002B5044503A20BE
:106840004445414354002B435245473A20300022EF
:106850002C2236383637220D0041542B43495053F1
:10686000544152543D22544350222C220041542B77
:10687000434C504F52543D22544350222C22363820
:106880003637220D0041542B43494653520D0041E7
:10689000542B434950484541443D310D0041542B50
:1068A00043494943520D00222C220041542B4353AB
:1068B00054543D2200220D0041542B434744434F82
:1068C0004E543D312C224950222C22002B434D4561
:1068D000204552524F520041542B43495053485582
:1068E000540D00495000534D53004D502D30205051
:1068F00041414C455254212121204352495449439E
:10690000414C20534F43204C4556454C204150505C
:10691000524F414348454420282575252520534F93
:106920004329004D502D302050415472756E6B201C
:10693000686173206265656E206F70656E656420A6
:106940002876616C6574206D6F6465292E0025754D
:1069500025250020534F433A20002575204B6D001C
:106960002575206D69000D496465616C2052616E6A
:1069700067653A20004368617267696E67205374E7
:106980006F70706564004368617267696E672C2080
:1069900048656174696E6700507265706172696EF6
:1069A00067004368617267696E6720446F6E6500B7
:1069B0004368617267696E672C20546F7070696EEE
:1069C00067206F6666004368617267696E67005092
:1069D0006572666F726D616E6365202D2000526175
:1069E0006E6765202D200053746F72616765202DDE
:1069F00020005374616E64617264202D2000202D8C
:106A0000204D53473A2000534D532046524F4D3AA4
:106A100020004D502D30205041004D502D3020632E
:106A200025642C33000D00222C31350D0041542BF0
:106A3000435553443D312C22004D502D30206333BB
:106A40002C302C25642C25642C2573004D502D30C2
:106A50002063312C302C25642C25642C2564004DBA
:106A6000502D302061004D502D3020004D502D53C1
:106A7000203020004D502D302045540025732C250A
:106A8000642C25642C25642C25642C25642C256419
:106A90002C004D502D3020670025642C25642C25BA
:106AA000642C25642C25642C25642C25642C256CF1
:106AB000752C25642C256C752C25642C25642C25BF
:106AC000642C2564004D502D3020440025642E2573
:106AD000642E25642C25732C25642C25642C2573A9
:106AE000004D502D30204600256400302C302C0005
:106AF00025642E25642C25642C004D502D30205704
:106B0000002C25642C25642C25642C2564004D5014
:106B10002D30204C0025642C25752C25642C2564F3
:106B20002C25642C25642C25642C25642C25642CB0
:106B300025640025752C002C00706572666F726DDF
:106B4000616E63652C0072616E67652C0073746FF3
:106B5000726167652C007374616E646172642C00ED
:106B600073746F707065642C0068656174696E671A
:106B70002C00707265706172652C00646F6E652CFC
:106B800000746F706F66662C006368617267696E6F
:106B9000672C0025642C25732C25642C25642C007F
:106BA0004D502D3020530020004D502D43203020DB
:106BB000000D0A004D502D3020454D001A00415463
:106BC0002B43495053454E440D004F564D532046DC
:106BD00069726D776172652076657273696F6E3A5E
:106BE0002025642E25642E25640050455200524114
:106BF0004E0053544F00535441000D2025753A2543
:106C0000640046656174757265733A000D204E45E7
:106C1000542053746174653A307825303278000D11
:106C20002047524E204C65643A2564000D205245A1
:106C300044204C65643A256400444941473A000DBC
:106C400020506172616E6F69643A2573000D2049AE
:106C5000503A2573005365727665723A000D2047ED
:106C6000534D2F475052533A204E6F7420636F6E2E
:106C70006E65637465642028307825303278290089
:106C80000D2047534D3A204F4B0D205365727665CA
:106C9000723A204E6F7420636F6E6E656374656424
:106CA000000D20475052533A204F4B0D2053657230
:106CB0007665723A20436F6E6E6563746564204F2B
:106CC0004B000D2050617373776F72643A25730027
:106CD0000D20557365723A2573000D2041504E3AD0
:106CE000257300475052533A000D204E6F74696669
:106CF00069636174696F6E733A2573000D20556E78
:106D00006974733A2573000D2056656869636C6574
:106D100049443A2573004D6F64756C653A000D2047
:106D200025753A00506172616D733A002C004D6F09
:106D300064756C652070617373776F72643A202597
:106D4000730052656769737465726564206E756D52
:106D50006265723A20257300414C4552542121212D
:106D600020435249544943414C20534F43204C4502
:106D700056454C20415050524F41434845442028ED
:106D80002575252520534F432900257525250020ED
:106D90000D534F433A20002575204B6D002575207B
:106DA0006D6900200D496465616C2052616E6765F4
:106DB0003A20004E6F74206368617267696E6700E5
:106DC0004368617267696E672053746F70706564A1
:106DD000004368617267696E672C20486561746959
:106DE0006E67004368617267696E672C2050726538
:106DF000706172696E67004368617267696E6720CF
:106E0000446F6E65004368617267696E672C205439
:106E10006F7070696E67206F6666004368617267A5
:106E2000696E6700506572666F726D616E63652092
:106E30002D200052616E6765202D200053746F7203
:106E4000616765202D20005374616E646172642057
:106E50002D20001A00220D0A0041542B434D4753A8
:0D6E60003D2200256C692E2530366C69003E
:026E6E006EDADA
:106E7000CED9E840E8403F0BE5D91BDA010EAFD987
:106E8000EF50F00BE8380F0B006EC1D9030B100D5B
:106E9000F3500010D7D9E66E010EA8D929DA1BE20B
:106EA00000500108000E015416E2060E036E53DA7C
:106EB000C00B03C0E7FFE75204E0E8427F0BE706A0
:106EC000FCE1026E010E8BD9EF500F0B040DF35055
:106ED0000210B8D901D03D0EE66E020E87D908DA4D
:106EE00009E200500208000E015404E234DA3F0BBC
:106EF000A9D901D03D0EE66E030E78D9ECD1CFD9D9
:106F0000A9D921E28DD901E3DB2AC0D916E1ED50E0
:106F100014E1030EE66EE66A71D9B4D901E6DFD951
:106F20000AE278D9EDD901E3DB2A19DADF2A010E6A
:106F3000F4E3DB2AF2D7DE6ADD6A020EDB2A030EF7
:106F4000DFE3DB2ADDD731DA013420E2005000082C
:106F5000000E01541BE2B1D9C7D904E6030E005C50
:106F6000000E015804E282D9F7E3DB2AF5D702DAF2
:106F700089D901E6B4D90AE24DD9C2D901E3DB2AA5
:106F8000EED9DF2A010EF4E3DB2AF2D7F90EDBCFCC
:106F9000E9FFFA0EDBCFEAFFEF6A040EE15C02E2E2
:106FA000E16AE552E16E97D17AD954D91BE238D91A
:106FB00001E3DB2A6BD910E1ED500EE1030EE66E22
:106FC000E66A1CD95FD901E68AD904E2CCD9FAE392
:106FD000DB2AF8D7DE6ADD6A020EDB2A030EE5E360
:106FE000DB2AE3D7E2D901341AE200500008000E90
:106FF000015415E262D978D904E6030E005C000E54
:10700000015804E233D9F7E3DB2AF5D7B3D93AD9EB
:1070100001E665D904E2A7D9FAE3DB2AF8D7040E22
:10702000E15C02E2E16AE552E16E55D18FD9010ED1
:10703000D6D8EF380F0B006EEAD8040DF3500010CD
:1070400038D989D9E840E8403F0B006E010EC7D817
:10705000EF38F00B0010E66E010EC8D8030EBFD853
:10706000EFCF00F078D9400DF350C00B0010E66E62
:10707000020EBCD830D16AD9070EE126050EDB6AB4
:10708000060EDB6AC4D801E197D0030EDB6A040E5A
:10709000DB6A010EDB6A020EDB6A3AD9D890015036
:1070A00001E61DD94AE2B3D848E0DF6AB0D82FE044
:1070B000DF502DE1FD0EDBCFE9FFDB2AFE0EDBCF3B
:1070C000EAFF01E3DB2AEFCFDFFF2B0EDF5C05E3F6
:1070D000DF507A0802E3000E01D0010E000902E041
:1070E000000E09D02B0EDF5CF76A310FF66E940E9E
:1070F000F7220800F550DF6EDF50D8E0240EDF5C89
:1071000002E1000E02D03D0EDF5CDF6ECFD77FD8EC
:107110000CE0030EDB2A040E01E3DB2ADF5007E05C
:10712000DF04E66ED5D81BD902D0D2D8EF6A010EA3
:10713000DB2A020EB2E3DB2AB0D7D950030FE96E87
:10714000DACFEAFFEE50ED109DE0F7D86FDFE552A1
:10715000E552E552E552010EDB6A020EDB6AD8D831
:10716000030EDBCF02F0040EDBCF03F00206000EAD
:10717000035A01500318E8AE02D0033404D0025081
:10718000005C0350015801E37DD701D9F9D8FB0E0B
:10719000DBCFE9FFDB2AFC0EDBCFEAFF01E3DB2AD2
:1071A000DED8050EDB2A060E01E3DB2A010EDB2A00
:1071B000020ED5E3DB2AD3D7B2D8EF6A050EDBCFB8
:1071C00000F0060EDBCF01F000C0F3FF01C0F4FFBA
:1071D000070EE15C02E2E16AE552E16E7CD0E76E07
:1071E000DDD8E750E926000EEA221200E76E97D8B4
:1071F000E750E926000EEA22AFEF39F09ED837DEDD
:10720000006E060EE15E0050DE6ADD6A1200C6D82E
:10721000EF501200DECFE9FFDDCFEAFFC0EF39F01B
:1072200085D8FD0EDB500024E96EFE0EDB500120F8
:10723000EA6EEF50E66EDFCFE9FFDF2A010EDBCF0B
:10724000EAFF1200F76AF00FF66E930EF7220800BD
:10725000F55012006BD8FB0EDBCF02F0FC0EDBCF3B
:1072600003F00250005C035001581200020EDBCF05
:10727000E9FF030EDBCFEAFF9DD8EF6A020EDB2A9F
:10728000030E120092D8D8900150120093D867D8FC
:10729000D9CFE9FFDACFEAFF030EEE18120056D875
:1072A000040EE126DE6ADD6A020EDB6A030EDB6A8B
:1072B0001200E66E34D8AFEF39F0D9CFE9FFDACF5C
:1072C000EAFF020EEECFDBFF030EEDCFDBFF120075
:1072D0005ED8DAEF39F0E552E7CFD9FF1200040E9D
:1072E000005C000E0158120021D8D8900150120005
:1072F000F90EDBCF00F0FA0EDBCF01F00134120003
:10730000F90EDBCFE9FFDB2AFA0EDBCFEAFF120032
:10731000010EDBCF00F0020EDBCF01F01200FB0EFE
:10732000DBCFE9FFFC0EDBCFEAFF1200020EDBCF62
:1073300000F0030EDBCF01F01200EA0EE66E080E3D
:10734000E66EE60EE66E080EE66E1200D9CFE6FF98
:10735000E1CFD9FF1200020E42DFEF501200E552DA
:10736000E750EF6E120056DF10EC1AF0E552DF2AFC
:10737000010E1200DECFE6FFDDCFE6FFFEEF38F0B4
:10738000EA0EE926080EEA22EF50E66E1200010E20
:10739000DBCFE9FF020EDBCFEAFF1200FD0EDBCFF1
:1073A000E9FFFE0EDBCFEAFF1200DECF00F0DDCFFB
:0E73B00001F01200E60EE926080EEA22120095
:0273BE00506518
:1073C000726D697373696F6E2064656E69656400C0
:1073D000596F75722070686F6E65206861732062E6
:1073E00065656E2072656769737465726564206196
:1073F0007320746865206F776E65722E004D6F6420
:10740000756C652070617373776F72642068617347
:10741000206265656E206368616E6765642E00504A
:107420006172616D65746572732068617665206252
:1074300065656E207365742E0046656174757265AE
:1074400020686173206265656E207365742E004844
:107450006F6D656C696E6B206163746976617465CC
:10746000640056656869636C65206C6F636B20729D
:1074700065717565737465640056656869636C65EC
:1074800020756E6C6F636B207265717565737465C2
:10749000640056616C6574206D6F6465207265715F
:1074A0007565737465640056616C6574206D6F64F6
:1074B000652063616E63656C2072657175657374B8
:1074C000656400436861726765206D6F6465206361
:1074D00068616E67652072657175657374656400B7
:1074E000436861726765207374617274207265719C
:1074F00075657374656400436861726765207374B1
:107500006F7020726571756573746564005472756F
:107510006E6B20686173206265656E206F70656EAA
:107520006564202876616C6574206D6F6465292E12
:1075300000436172206C6F636174696F6E3A0D680D
:107540007474703A2F2F6D6170732E676F6F676C54
:10755000652E636F6D2F6D6170732F6170692F736E
:1075600074617469636D61703F7A6F6F6D3D313521
:107570002673697A653D353030783634302673634A
:10758000616C653D322673656E736F723D66616C2A
:107590007365266D61726B6572733D69636F6E3AD8
:1075A000687474703A2F2F676F6F2E676C2F70425C
:1075B0006358372537430052454749535445523F96
:1075C00000000000000000000000000000000000BB
:1075D0000000524547495354455200000000000046
:1075E00000000000000000000000000000504153B7
:1075F000533F0000000000000000000000000000F9
:107600000000000000000000504153532000000023
:10761000000000000000000000000000000000006A
:107620000000004750530000000000000000000070
:1076300000000000000000000000000000005354A3
:1076400041540000000000000000000000000000A5
:10765000000000000000000000504152414D533F27
:10766000000000000000000000000000000000001A
:1076700000000000504152414D5320000000000026
:107680000000000000000000000000000000004DAD
:107690004F44554C453F0000000000000000000032
:1076A000000000000000000000004D4F44554C4514
:1076B00020000000000000000000000000000000AA
:1076C0000000000000475052533F0000000000003F
:1076D00000000000000000000000000000000000AA
:1076E000475052532000000000000000000000003E
:1076F0000000000000000000000000534552564505
:10770000523F0000000000000000000000000000E8
:107710000000000000005345525645522000000072
:107720000000000000000000000000000000000059
:107730000044494147000000000000000000000034
:107740000000000000000000000000004645415419
:10775000555245533F0000000000000000000000AB
:1077600000000000000000464541545552452000ED
:107770000000000000000000000000000000000009
:107780000000484F4D454C494E4B20000000000082
:10779000000000000000000000000000004C4F430B
:1077A0004B2000000000000000000000000000006E
:1077B0000000000000000000554E4C4F434B2000DD
:1077C00000000000000000000000000000000000B9
:1077D00000000056414C455420000000000000000D
:1077E0000000000000000000000000000000554EF6
:1077F00056414C45542000000000000000000000ED
:107800000000000000000000004348415247454D81
:107810004F44452000000000000000000000000070
:107820000000000043484152474553544152540020
:107830000000000000000000000000000000004305
:10784000484152474553544F50000000000000008B
:107850000000000000000000000056455253494F50
:107860004E000000000000000000000000000000CA
:107870000000000000524553455400000000000085
:1078800000000000000000000000000000000000F8
:1078900000000000000000000000000000000000E8
:0B78A0000000000000000000000000DD
:0478AC00219E05D044
:1078B000219E29AE02D0296C218E29C023F0226A94
:1078C000336A326A860E246E256A27EF3EF0219EC7
:1078D0000CD0219E29AE09D0266C271E281E291EF9
:1078E000E86A272228222922218E29C023F028C0D5
:1078F00022F027C033F026C032F09E0E246E256A97
:1079000027EF3EF0216A63EC3EF07BEC3EF021B6BF
:107910000BEF3EF021A205D021BA0BEF3EF012EFA3
:107920003EF021BA1EEF3EF021A005D021B80BEFAA
:107930003EF01EEF3EF021B812EF3EF0256A7F0EBA
:107940002A24246EE86A25222F50245EE86A255AEC
:107950001A0E306E2A6A326A336A226A236A2C50FF
:10796000275E2D50285A2E50295A000E2A5A09E710
:107970002C5027262D5028222E502922000E2A2254
:1079800001D0328AD8902736283629362A36D89020
:107990003236333622362336302EE1D7295028109E
:1079A0002710D8A4328A27EF3EF0216A63EC3EF01C
:1079B0007BEC3EF021B60BEF3EF021A205D021B8C2
:1079C0000BEF3EF012EF3EF021AA05D021B00BEFF5
:1079D0003EF012EF3EF021B002D021A802D01EEFFF
:1079E0003EF0256A2F502A24246EE86A25227E0E56
:1079F000245EE86A255A326A336A226A236A2E5064
:107A00002902F4CF23F0F3CF22F02D502902F350B6
:107A10003326F4502222000E23222E502802F35047
:107A20003326F4502222000E23222C502902F35038
:107A30003226F4503322000E222223222D50280217
:107A4000F3503226F4503322000E222223222E50ED
:107A50002702F3503226F4503322000E2222232232
:107A60002C502802F4503226000E332222222322E8
:107A70002D502702F4503226000E332222222322D8
:107A800027EF3EF0206A2EAE48EF3DF02E6C201E10
:107A900029AE4DEF3DF0296C201E43EC4BF029BE82
:107AA00057EF3DF020AE000C296C256C000C20BE79
:107AB00054EF3DF02188FF0C206A2EAE65EF3DF0BB
:107AC0002D6C2E1EE86A2E22201E29AE6DEF3DF091
:107AD000286C291EE86A2922201EDFEC4AF029BE04
:107AE0007DEF3DF020AE000C286C291EE86A2922AB
:107AF000246C251EE86A2522000C20BE74EF3DF0A0
:107B00002188FF0C206AE86A2EAE8FEF3DF02B6CC7
:107B10002C1E2D1E2E1E2C222D222E22201E29AE82
:107B20009AEF3DF0266C271E281E291E27222822A8
:107B30002922201EBBEC4AF029BEB1EF3DF020AE59
:107B4000000C266C271E281E291EE86A27222822E0
:107B50002922226C231E241E251E232224222522B4
:107B6000000C20BEA1EF3DF02188FF0C28C032F0B0
:107B700028502D02F4CF27F0F3CF26F029502E0203
:107B8000F4CF29F0F3CF28F02D02F3502726F4503C
:107B90002822E86A292232502E02F3502726F45078
:107BA0002822E86A2922000C216A63EC3EF021B603
:107BB000DEEF3DF021A20FD021B407D07F0E296E59
:107BC000FF0E286E276E266E25D0800E296E01D0FE
:107BD000296A000EF6D721B0FBD7266A9F0E2A60CD
:107BE000EBD77E0E2A64F4D79E0E2A5C07E0D8906D
:107BF00029322832273226322A2AF6D721A40AD05F
:107C0000266C271E281E291EE86A272228222922E0
:107C100029AEDED712007F0E2A6EFF0E296E286E67
:107C2000276E12007F0E21BEFF0E2A6E02D07F0E3D
:107C30002A6E800E296E286A276AF3D721AE04D0F7
:107C4000800E2A6E296AF7D72A6A296AF4D7235048
:107C5000221033103210F8E025BEF0D723BE0CD02E
:107C600024502510EBE0D8903236333622362336B6
:107C70002406D8A02506F2D72550D4E12428D2E046
:107C800032AE11D07F0E321402E133A00CD0332A71
:107C9000E86A2222232207E3D880233222323332B9
:107CA000242A2428BFE02450C9E033C027F022C092
:107CB00028F02334296E24302A6E29322A9E21BED0
:107CC0002A8E11EF3EF029362A3602E32184217EE6
:107CD00006E121802A6A296A286A276A12002A286E
:107CE00003E0D88029321200D890293202E12182A3
:107CF0001200218612002E362F3602E3218C217EBF
:107D000006E121882F6A2E6A2D6A2C6A12002F281C
:107D100003E0D8802E321200D8902E32EAE1218A78
:107D2000120029C033F028C032F028502D02F4CFC1
:107D300027F0F3CF26F029502E02F4CF29F0F3CF0D
:107D400028F02D02F3502726F4502822E86A292231
:107D500032502E02F3502726F4502822E86A2922B6
:107D60002EAEB7EF3EF03250285E3350295A33AE74
:0C7D7000000C2D50285E2E50295A000CEB
:047D7C00FB0EE3CF48
:107D8000F6FFFC0EE3CFF7FFFD0EE3CFF8FFFE0E8C
:107D9000E3CFE9FFFF0EE3CFEAFFF90EE35003E183
:107DA000FA0EE35009E0F90EE30602E2FA0EE306EA
:107DB0000900F550EE5CF1E01200D9CFE6FFDACF12
:107DC000E6FFFA0EE3CFD9FFFB0EE3CFDAFFFC0E9E
:107DD000E3CFE9FFFD0EE3CFEAFFE9CFF3FFEACF00
:107DE000F4FFF80EE35003E1F90EE35008E0F80E5B
:107DF000E30602E2F90EE306DECFEEFFF2D7FF0E56
:107E0000E3CFDAFFE552FF0EE3CFD9FFE5521200D0
:107E1000FE0EE3CFE9FFFF0EE3CFEAFFE9CFF3FF6A
:107E2000EACFF4FFFB0EE35003E1FC0EE35009E060
:107E3000FB0EE30602E2FC0EE306FD0EE350EE6EDF
:107E4000F1D71200D9CFE6FFDACFE6FFFA0EE3CF83
:107E5000D9FFFB0EE3CFDAFFFC0EE3CFE9FFFD0E07
:107E6000E3CFEAFFE9CFF3FFEACFF4FFEE66FED7F8
:107E7000ED52DFCFEEFFDE66FCD7FF0EE3CFDAFF79
:107E8000E552FF0EE3CFD9FFE5521200FB0EE3CF20
:107E9000F6FFFC0EE3CFF7FFFD0EE3CFF8FFFE0E7B
:107EA000E3CFE9FFFF0EE3CFEAFFE9CFF3FFEACF2D
:107EB000F4FFEE66FED7ED520900F5CFEFFFEE6658
:107EC000FBD71200D9CFE6FFDACFE6FFFA0EE3CFF9
:107ED000D9FFFB0EE3CFDAFFFC0EE3CFE9FFFD0E87
:107EE000E3CFEAFFDE50EF5C02E1EE66FBD7F36E14
:107EF000FF0EE3CFDAFFE552FF0EE3CFD9FFE552E5
:107F0000F3501200D9CFE6FFDACFE6FFFA0EE3CF47
:107F1000D9FFFB0EE3CFDAFFFC0EE3CFE9FFFD0E46
:107F2000E3CFEAFFE9CFF3FFEACFF4FFDECFEFFFC5
:107F3000EE66FCD7FF0EE3CFDAFFE552FF0EE3CF8C
:107F4000D9FFE5521200FB0EE3CFF6FFFC0EE3CFA4
:107F5000F7FFFD0EE3CFF8FFFE0EE3CFE9FFFF0EC4
:107F6000E3CFEAFFE9CFF3FFEACFF4FF0900F5CF53
:107F7000EFFFEE66FBD71200FE0EE3CFE9FFFF0E28
:107F8000E3CFEAFFF36AF46AEE5203E0F34AF42A1D
:107F9000FBD71200FF0EE3CFF8FFE552FF0EE3CF51
:107FA000F7FFE552FF0EE3CFF6FFE552E66AE66A19
:107FB000E66A0900F55209E0FD0EE32A05E1FE0E2E
:107FC000E32A02E1FF0EE32AF4D7FD0EE3CF27F008
:107FD000FE0EE3CF28F0FF0EE3CF29F01200D9CF39
:107FE000E6FFDACFE6FFFA0EE3CFD9FFFB0EE3CFD1
:107FF000DAFFFC0EE3CFE9FFFD0EE3CFEAFFF80E58
:10800000E35003E1F90EE3500AE0F80EE30602E262
:10801000F90EE306DE50EF5C02E1EE66F0D7F36E98
:10802000FF0EE3CFDAFFE552FF0EE3CFD9FFE552B3
:10803000F3501200D9CFE6FFDACFE6FFFA0EE3CF16
:10804000D9FFFB0EE3CFDAFFFC0EE3CFE9FFFD0E15
:10805000E3CFEAFFE9CFF3FFEACFF4FFF80EE350F6
:1080600003E1F90EE3500BE0F80EE30602E2F90E2D
:10807000E306DECFEFFFEE66F1D7DD52EFD7FF0E5E
:10808000E3CFDAFFE552FF0EE3CFD9FFE55212004E
:10809000FE0EE3CFF3FFFF0EE3CFF4FFFB0EE3CFC3
:1080A000F6FFFC0EE3CFF7FFFD0EE3CFF8FFF3CFB3
:1080B000E9FFF4CFEAFF0900F5500CE0F550EF5C62
:1080C00002E1EE52F8D7EF5203E0F34AF42AE6D782
:1080D000F36AF46A1200FE0EE3CFE9FFFF0EE3CF6E
:1080E000EAFFE9CFF3FFEACFF4FF610EEF5C05E6AC
:1080F0007B0EEF5C02E7DF0EEF16EE52F6E11200A8
:10810000D9CFE6FFE1CFD9FF0A0EE126020EDB6AE6
:10811000030EDB6A040EDB6A050EDB6A1CD9EF6A0C
:108120001AD9EE52EF6A2FD9080EE9CFDBFF090EFC
:10813000EACFDBFFDE6ADD6A2DD904E6000E005CC3
:10814000010E015808E201D9DFCFEFFFDF2A010E4F
:10815000F3E3DB2AF1D7DE6ADD6A1CD904E6000E00
:10816000005C010E01586BE2F0D8EF50E66ED9507A
:10817000060F01D9060EDBCF02F0070EDBCF03F0AE
:10818000020EDB500224006E030EDB500320040EAF
:10819000DBCF06F0050EDBCF07F0F90EDB5006242F
:1081A000E96EFA0EDB500720EA6EEF50046E056AA6
:1081B00000500424E66ED950020FDDD8020EDBCF4A
:1081C00002F0030EDBCF03F0080EDB500224E96E51
:1081D000090EDB500320EA6EEF50E66EB6D8E5528A
:1081E000E750EF6E020EDBCF00F0030EDBCF01F0A5
:1081F000080EDB500024E96E090EDB500120EA6E08
:10820000060EDBCFEFFF040EDB2ADBCF00F0050EFE
:1082100001E3DB2ADBCF01F0A5D8E8AE02D00334BE
:1082200004D00250005C0350015804E3040EDB6AE2
:10823000050EDB6ADF2A010E90E3DB2A8ED70A0ED9
:10824000E15C02E2E16AE552E16EE552E7CFD9FF77
:108250001200D9CFE6FFE1CFD9FF080EE1267BD887
:10826000040EEFCFDBFF77D8EE52050EEFCFDBFF2A
:108270008AD8020EE9CFDBFF030EEACFDBFFDE6A0E
:10828000DD6ADECF00F0DDCF01F06CD8E8AE02D0C1
:10829000033404D00250005C0350015837E2040E4E
:1082A000DB2ADB5046D8060EEFCFDBFF050EDBCF17
:1082B000E7FF060EDB50E726050EE7CFDBFFDB50BE
:1082C00038D8070EEFCFDBFF040EDB5032D8070E95
:1082D000DBCFEFFF050EDB502CD8060EDBCFEFFF18
:1082E000070EDBCFE6FF060EDB50E552E72421D870
:1082F000EFCF02F0F90EDBCF00F0FA0E52D80250A9
:10830000EF1ADF2A010EBDE3DB2ABBD724D8040E07
:10831000DBCFEFFF20D8EE52050EDBCFEFFF080ECC
:10832000E15C02E2E16AE552E16EE552E7CFD9FF96
:108330001200E76E020EDBCFE9FF030EDBCFEAFF90
:10834000E750E926000EEA221200080EDBCF00F00B
:10835000090ED1EF41F0FD0EDBCFE9FFFE0EDBCFC2
:10836000EAFF1200F70EDBCF02F0F80EDBCF03F0CE
:10837000015003181200E96EDACFEAFFE552E75028
:10838000EE6EED6A1200FB0EDBCFE9FFFC0EDBCFD9
:10839000EAFF1200DECF00F0DDCF01F0D8900150EF
:1083A0001200DBCF01F0DE500024E96EDD50012029
:0483B000EA6E12005F
:0C83B400FF0012004ED9E652DF6A7C0E7A
:1083C000CA6ECC6ACB687A0EDF5C05E29EA2FED74D
:1083D0009E92DF2AF8D7E55231D13DD9FE0EDB500F
:1083E000000804E2E9DFFE0EDB06F8D727D1D9CF7B
:1083F000E6FF24D1D9CFE6FF21D181B005D081801D
:10840000050EE66EEADFE55281900C0EE66EE5DFC2
:10841000E552818012001FD90C0EE126D950FB0FC6
:10842000E96EFF0EDA20EA6ED890030EEB50000AD8
:1084300008E6000EEE5C000EEE58000EEE58000E40
:10844000EE5827E2F90EDBCFE9FFDB2AFA0EDBCF8D
:10845000EAFF01E3DB2A2D0EEF6EFB0EDBCF00F00F
:10846000FC0EDBCF01F0FD0EDBCF02F0FE0EDBCF0A
:1084700003F0001E011E021E031EFB0E00C0DBFFE8
:10848000FC0E01C0DBFFFD0E02C0DBFFFE0E03C0D1
:10849000DBFFFB0EDBCF08F0FC0EDBCF09F0FD0E9F
:1084A000DBCF0AF0FE0EDBCF0BF0CCD869EC3CF052
:1084B00027C004F028C005F029C006F02AC007F044
:1084C0002C6A2D6A2E6A450E2F6E82EC3CF027C076
:1084D00000F028C001F029C002F02AC003F02C6A85
:1084E0002D6A610E2E6E450E2F6E82EC3CF027C079
:1084F000DEFF28C0DEFF29C0DEFF2AC0DDFFDD521F
:10850000DD52DECF27F0DECF28F0DECF29F0DDCF41
:108510002AF0DD52DD52D4EC3DF0040E26C0DBFF24
:10852000050E27C0DBFF060E28C0DBFF070E29C0A3
:10853000DBFF040EDBCF08F0050EDBCF09F0060EE3
:10854000DBCF0AF0070EDBCF0BF0400E2B6E420E96
:108550002C6E0F0E2D6E2E6A75D883EC4AF022C059
:1085600008F023C009F024C00AF025C00BF0D9CFD1
:10857000E9FFDACFEAFFEECF04F0EECF05F0EECF61
:1085800006F0EFCF07F02C6A240E2D6E740E2E6EBF
:10859000490E2F6E04C027F005C028F006C029F050
:1085A00007C02AF0D5EC3CF0D4EC3DF000010850B7
:1085B000265C006E09502758016E0A502858026E3A
:1085C0000B502958036E080E00C0DBFF090E01C0D6
:1085D000DBFF0A0E02C0DBFF0B0E03C0DBFFD9502E
:1085E000080F20D8D950040F1DD8630E006E6E0EF0
:1085F000016E026A00C0E6FFE66E02C0E6FFF90EF9
:10860000DBCFE6FFFA0EDBCFE6FF04EC49F0036EAA
:108610000D0EE15E03500C0EE15C02E2E16AE552F0
:10862000E16E0CD0E96EDACFEAFFEECFE6FFEECFD7
:10863000E6FFEECFE6FFEFCFE6FF1200E552E7CF11
:10864000D9FF120008C026F009C027F00AC028F0A0
:108650000BC029F01200D9CFE6FFE1CFD9FF1200FD
:10866000FF0EE3CFEAFFE552FF0EE3CFE9FFE5524D
:10867000E66AE66AD9CFE6FFDACFE6FFFC0EE12430
:10868000D96EFF0EE220DA6EE66AE66AE66A200E2E
:10869000EF5C06E0090EEF5C03E0EF6603D03FD02D
:1086A000EE50F5D72D0EEF5C03E1FF0EE32A03D069
:1086B0002B0EEF5C01E1EE502F0EEF6424D03A0E4A
:1086C000EF6021D0D890F90EE336FA0EE336FD0EB6
:1086D000DECFE3FFFE0EDDCFE3FFD890F90EE336E9
:1086E000FA0EE336D890F90EE336FA0EE336FD0EB5
:1086F000E350DE26FE0EE350DD22300EEE5CDE2679
:10870000000EDD22D9D7FF0EE3CFE8FFE85207E0E5
:10871000F90EE31EE32AFA0ED8B4E306E31EE5528F
:10872000E552E552FF0EE3CFDAFFE552FF0EE3CF4D
:10873000D9FFE552E1CFE9FFE2CFEAFFED52ED527A
:10874000EECFF3FFEFCFF4FF1200FF0EE3CFEAFF0F
:10875000E552FF0EE3CFE9FFE552E66AE66AE66A14
:10876000E66AD9CFE6FFDACFE6FFFA0EE124D96E4A
:10877000FF0EE220DA6EE66AE66AE66AE66AE66A12
:10878000200EEF5C06E0090EEF5C03E0EF6603D01D
:108790006BD0EE50F5D72D0EEF5C03E1FF0EE32A10
:1087A00003D02B0EEF5C01E1EE502F0EEF6444D0AE
:1087B0003A0EEF6041D0D890F50EE336F60EE33670
:1087C000F70EE336F80EE336FB0EDECFE3FFFC0ECA
:1087D000DECFE3FFFD0EDECFE3FFFE0EDDCFE3FFD6
:1087E000DD52DD52D890F50EE336F60EE336F70E85
:1087F000E336F80EE336D890F50EE336F60EE336A0
:10880000F70EE336F80EE336FB0EE350DE26FC0EE1
:10881000E350DE22FD0EE350DE22FE0EE350DD22A9
:10882000DD52DD52300EEE5CDE26000EDE22DE2250
:10883000DD22DD52DD52B9D7FF0EE3CFE8FFE8526B
:1088400013E0F50EE31EF60EE31EF70EE31EF80E20
:10885000E31EF50EE32A08E1F60EE32A05E1F70E22
:10886000E32A02E1F80EE32AE552E552E552E55229
:10887000E552D9CFE9FFDACFEAFFEECF26F0EECF0F
:1088800027F0EECF28F0EFCF29F0FF0EE3CFDAFF8D
:10889000E552FF0EE3CFD9FFE552E552E552120053
:1088A000FE0EE3CFFEF4FF0EE3CFFFF41200FFC491
:1088B00029F0FEC428F0350E2D6E450E2E6EB6EC56
:1088C0003DF0262AE86A2722279E27C0FFF426C00B
:0C88D000FEF4FEC4F3FFFFC4F4FF12002E
:0488DC001200D9CFDE
:1088E000E6FFE1CFD9FF040EE126A66AFE0EDB50BB
:1088F000E66ED950020FB0D8020EDBCF2DF0030E7A
:10890000DBCF2EF0B6EC3DF0020E26C0DBFF030EEF
:1089100027C0DBFF020E030EAAD8020EDBCF00F049
:10892000030EAFD8C1D804E6200E005C000E01583B
:108930000AE2A680B0D8A8CFEFFFA92ADF2A010E4D
:10894000F1E3DB2AEFD7DD0E006E090E016E00C0E9
:10895000F3FFF46E040EE15C02E2E16AE552E16EBF
:10896000E552E7CFD9FF1200D9CFE6FFE1CFD9FF1B
:10897000050EE126DE6ADD6A200EE66EE66AFC0E72
:10898000DBCFE6FFFD0EDBCFE6FFDD0EE66E090E68
:10899000E66E1AEC40F0006E060EE15E0050090132
:1089A000FC6BFE0EDB50E66ED950030F55D8030E5C
:1089B000DBCF2DF0040EDBCF2EF0B6EC3DF0030E36
:1089C00026C0DBFF040E27C0DBFF030EDBCF00F069
:1089D000040E4DD8030EDBCF00F0040E52D864D83D
:1089E00004E6200E005C000E01582CE2FE0EDB5067
:1089F000200DF3CF02F0F4CF03F0000E0226000E9C
:108A00000322DE500224006EDD500320016E005070
:108A1000A96EA66AA6843FD8EF50A86E020EF2CFC8
:108A2000DBFFF29E550EA76EAA0EA76EA682020E5F
:108A3000DB50F26EA6B2FED7A694DF2A010ECFE37A
:108A4000DB2ACDD7050EE15C02E2E16AE552E16E78
:108A5000E552E7CFD9FF1200E96EDACFEAFFE5521F
:108A6000E750EE6EED6A200E286E296A1200DBCF09
:108A700001F001C000F0016A0050AA6EFF0EE76E1F
:108A80001200DBCF01F0E7500016016A0050A96E1A
:108A9000DE6ADD6A1200DECFE9FFDDCFEAFFDD0E20
:108AA000E926090EEA221200DECF00F0DDCF01F048
:068AB000D89001501200F5
:0A8AB600D9CFE6FFE1CFD9FF040E8F
:108AC000E126DF6A080EDF5C09E2DF50EA6ACC0FBC
:108AD000E96E080EEA22EF6ADF2AF4D7080EDF6E8D
:108AE000100EDF5C20E2080EDF5C180FE66E6FEC04
:108AF00044F0E552F3CF00F0F4CF01F000C0E6FF00
:108B000001C0E6FF30EC43F0E552E552F350E66E6B
:108B1000DF50EA6ACC0FE96E080EEA22E552E75010
:108B2000EF6EDF2ADDD7806A0F0EC16E9268FE0EEF
:108B3000936E870ED56E09EC48F06EEC44F05EEC57
:108B40002EF08FEC1FF00A0EE66EEDEC41F0E552D0
:108B5000E668E66ADFEC47F0E552E552E66A010EA8
:108B6000E66EDFEC47F0E552E55206EC48F00A0EFF
:108B7000E66EEDEC41F0E55200C9E6FF010EE66E4F
:108B8000DFEC47F0E552E55206EC48F0230EE66EC6
:108B9000EDEC41F0E552040001C9E6FF010EE66E7E
:108BA000DFEC47F0E552E55206EC48F0230EE66EA6
:108BB000EDEC41F0E552040002C9E6FF010EE66E5D
:108BC000DFEC47F0E552E55206EC48F0230EE66E86
:108BD000EDEC41F0E5520400E66A010EE66EDFECD2
:108BE00047F0E552E552E66AE66ADFEC47F0E55207
:108BF000E55206EC48F00A0EE66EEDEC41F0E55267
:108C000004000A0EE66E010EE66EDFEC47F0E55258
:108C1000E55206EC48F0010EDB6A0801080100513C
:108C2000200B05E1080108010051100B02E00BECDC
:108C300019F0080100B702D00EEC19F015EC32F073
:108C40000400D650DF6E4C0ED75C07E3D76AD66AB5
:108C500059EC1FF0EDEC31F00ED0010EDB50D75C7B
:108C60000AE0D750030B04E18EEC1FF00FEC32F05A
:108C7000010ED7CFDBFFD1D7040EE15C02E2E16A3F
:0C8C8000E552E16EE552E7CFD9FF12008B
:048C8C00080100914A
:108C90000083416B426B436B00950087009B0099FA
:108CA000C46BC56BC66B810EAF6EAC84949C948E06
:108CB0009F989F9AAC8AAB88AB8E9D889D8AF28ED6
:108CC000F28C1200AFD8080100A102D0000E17D01C
:108CD0009D984251EA6A010FE96E080EEA22FE0EE3
:108CE000DBCFEFFF0093412B400E415D01E100819E
:108CF000422B400E425D01E1426B9D88010E97D0F0
:108D0000400E0801415D04E2400ED880415512003A
:108D1000000C88D8080100A702D0000E20D09D9A30
:108D20000095C651EA6A440FE96E080EEA22EF5038
:108D3000E66EFD0EDBCFE9FFFE0EDBCFEAFFE5526C
:108D4000E750EF6EC407C45101E10087C62BC6513E
:108D500072D803E1015001E1C66B9D8A010E67D014
:108D60000801C45112005ED8E6529D50100B01E07C
:108D7000010E006E9E50100B01E0010E001419E070
:108D8000080100B314D04351EA6A010FE96E080EDE
:108D9000EA22EF50AD6E00B100914107415101E16F
:108DA0000083432B400E435D3BE1436B39D09D98DC
:108DB00037D09D50200B01E0010E006E9E50200B1D
:108DC00001E0010E00142CE0ABB404D0ABA207D03C
:108DD000AB98AB88AE50DF6E0801008B21D0080144
:108DE00000A504D0AE50DF6E00891AD000B518D0AF
:108DF00000990097C551EA6A440FE96E080EEA220D
:108E0000AECFEFFFC42BC45116D803E1015001E1EE
:108E10000085C52BC5510FD803E1015001E1C56B99
:108E2000E55205D0D9CFE6FFE1CFD9FF1200E552D8
:108E3000E7CFD9FF1200006E016A800E0018120001
:108E4000D9CFE6FFE1CFD9FF020EE126400EE66E54
:108E5000E66AE66A000EE66E040EE66E08EC3FF087
:108E6000006E050EE15E0050400EE66EE66AE66AB0
:108E7000400EE66E040EE66E08EC3FF0006E050E46
:108E800076D8000EE66E040EE66EDDEC3EF0006E67
:108E9000060E6DD8400EE66E040EE66EDDEC3EF07A
:108EA000006E060EE15E0050DE6ADD6ADECF00F085
:108EB000DDCF01F0D890015004E6400E005C000EBA
:108EC00001581DE2360E006EDECFE9FFDDCFEAFF6E
:108ED000000EE926040EEA220050EF1A5C0E006E26
:108EE000DECFE9FFDDCFEAFF400EE926040EEA22DD
:108EF0000050EF1ADF2A010ED9E3DB2AD7D746D874
:108F0000000EE66E040E4BD8FB0EDBCFE6FFFC0E28
:108F1000DBCFE6FFFD0EDBCFE6FFFE0E17D836D81F
:108F2000400EE66E040E3BD8100EE66EE66AF50EB5
:108F3000DBCFE6FFF60E0AD8020EE15C02E2E16A40
:108F4000E552E16EE552E7CFD9FF1200DBCFE6FF35
:108F500029D830D8F50EDBCFE6FFF60EDBCFE6FFE3
:108F6000B0EC01F0E552E552E552E5521200E15E47
:108F70000050F70EDBCFE6FFF80EDBCFE6FFF90E71
:108F8000DBCFE6FFFA0EDBCFE6FF120013D840EC92
:108F900000F0E552E552400EE66EE66A1200E66E1B
:108FA000D2EF47F007D883EC00F0006E060EE15ECA
:0E8FB00000501200800EE66E040EE66E1200F7
:028FBE00D9CF09
:108FC000E6FFE1CFD9FFFE0EDB50EA6AF40FE96E4F
:108FD000080EEA22FD0EDBCFEFFFDB50FF0812E1A7
:108FE000FD0EDB50040F006E010E005202E0A1D80E
:108FF000FEE18212FE0EDB50EA6AF60FE96E080E01
:10900000EA22EF6AE552E7CFD9FF12000801F86BB8
:109010001200CF0E8216B50ECD6E9F909D80CE6A47
:10902000CF6A12009EA06FD00801F83502E3F82B3A
:1090300069D0F85127E10501FF6B020EFF5D1FE2C9
:1090400070D8E66E61D8E552E750EF6E6AD805E158
:1090500062D810E06ED8FEE10DD063D8FF0806E1BB
:109060005AD802E066D8FEE1821206D054D802E057
:1090700060D8FEE1E81C82160501FF2BDED708014F
:109080001F0E03D0F80503E1F60EF86F3BD0F8078A
:109090000501FF6B020EFF5D35E236D8EFCF00F021
:1090A000000EE76E0018E8AE02D0003403D0E7509F
:1090B000D88000541BE2F8C829F0030E2E6E42EC53
:1090C0003DF0255009E105011FD8EF0624D802E044
:1090D00030D8FEE1821213D0040E0501FF25006E88
:1090E000010E00520AE025D8FEE107D00DD8EF505E
:1090F00006E111D802E01DD8FEE1E81C8216050148
:10910000FF2BC8D79E901200FF51EA6AF60FE96E56
:10911000080EEA221200040EFF25006E010E005216
:109120001200FF51EA6AF40FE96E080EEA22EF50CE
:0A9130001200E846FE0B00061200D4
:06913A004D502D302063B2
:1091400025642C30004D502D30206325642C312CAB
:10915000496E76616C69642073796E746178004D34
:10916000502D30206325642C312C4E6F207772698E
:1091700074652061636365737320746F2043414E8F
:10918000004D502D30206325642C312C50617261CC
:109190006D65746572206F7574206F662072616EE4
:1091A0006765004D502D30206325642C312C4361C0
:1091B0006E6E6F74206368617267652028636861F2
:1091C00072676520706F727420636C6F73656429B9
:1091D000004D502D30206325642C312C43616E6E80
:1091E0006F742073746F70206368617267652028E4
:1091F000636861726765206E6F7420696E2070729B
:089200006F67726573732900AA
:08920800D9CFE6FFDACFE6FF43
:10921000E1CFD9FFE2CFDAFFE652E652E652E6525C
:10922000D950F90F006EFF0EDA20016E020E00C059
:10923000DBFF030E01C0DBFF020EDBCFE6FF030EF8
:10924000DBCFE6FFF90EDBCFE6FFFA0EDBCFE6FF62
:10925000FB0EDBCFE6FFD950FC0FE66EFF0EDA20E7
:10926000E66E14EC28F0006E070EE15C02E2E16AA3
:10927000E552E16E0050F3CFDEFFF4CFDDFFFC0ED0
:10928000DBCFE9FFFD0EDBCFEAFFEF6ADECF00F0B8
:10929000DDCF01F000C0F3FF01C0F4FF040EE15C7C
:1092A00002E2E16AE552E16EE552E5CFDAFFE7CF8F
:0492B000D9FF1200D0
:0C92B4001E0EF66E000EF76E000EF86E37
:1092C00008010900F550E16F0900F550E26F03E174
:1092D000E16701D03DD00900F550DC6F0900F55081
:1092E000DD6F0900F550DE6F09000900F550E96EE9
:1092F0000900F550EA6E090009000900F550DF6F1A
:109300000900F550E06F09000900F6CFE3F8F7CF48
:10931000E4F8F8CFE5F8DCC8F6FFDDC8F7FFDEC8F3
:10932000F8FF0801DF5302E1E05307E00900F550C0
:10933000EE6EDF07F8E2E007F9D7E3C8F6FFE4C80E
:10934000F7FFE5C8F8FF0801E107000EE25BBFD7B1
:02935000120009
:0E93520041542B43534D494E533F0D0041549F
:109360002B4350494E3F0D0041542B4950523F3B37
:109370002B435245473D313B2B434C49503D313BFC
:109380002B434D47463D313B2B434E4D493D322CFF
:10939000323B2B435344483D313B2B4349505350C0
:1093A00052543D303B2B4349505153454E443D317F
:1093B0003B45300D0041542B434F50533D300D0081
:1093C00041540D004154480D0041542B4352454730
:1093D0003F3B2B4349505354415455533B2B43532C
:1093E000510D0041542B4950523D393630300D005B
:1093F0004142434445464748494A4B4C4D4E4F50E5
:109400005152535455565758595A616263646566B0
:109410006768696A6B6C6D6E6F7071727374757664
:109420007778797A303132333435363738392B2FF3
:10943000007C2424247D72737475767778797A7B26
:10944000242424242424243E3F40414243444546CE
:109450004748494A4B4C4D4E4F5051525354555624
:109460005724242424242458595A5B5C5D5E5F6091
:109470006162636465666768696A6B6C6D6E6F7064
:02948000710079
:0E948200D9CFE6FFDACFE6FFE1CFD9FFE2CF88
:10949000DAFFFB0EDBCF00F0FC0EDBCF01F00001AA
:1094A000800E01141AE1FB0EDBCFE9FFFC0EDBCFCF
:1094B000EAFFEECFF3FFEDCFF4FFEE2A000EEF222E
:1094C000F3CFE9FFF4CFEAFFFD0EDBCFEFFFEF5064
:1094D000016AF36E01C0F4FF10D0FB0EDB50FE08F2
:1094E00006E1FD0EDBCFE6FF35EC4BF005D0FD0EBF
:1094F000DBCFE6FF03EC00F0E552E552E5CFDAFF03
:06950000E7CFD9FF1200C5
:0A95060026502B02F3CF22F0F4CF21
:1095100023F02C02F3502326000EF420246E265054
:109520002D02F3502426000EF420256E26502E0224
:10953000F350252627502B02F3502326F4502422E3
:10954000000E252227502C02F3502426F450252209
:1095500027502D02F350252628502B02F3502426A5
:10956000F450252228502C02F350252629502B0296
:06957000F3502526120055
:0A957600256A246A236A226A200E87
:10958000E76ED890263627362836293622362336F7
:10959000243625362B50225C2C5023582D5024582D
:1095A0002E50255809E32B50225E2C50235A2D5063
:0E95B000245A2E50255A262AE72EE4D7120000
:0295BE00256A1C
:1095C000246A100EE76ED8902836293624362536C0
:1095D0002D50245C2E50255805E32D50245E2E502E
:0A95E000255A282AE72EF0D71200C2
:0695EA00F36AF46AFF0EB3
:1095F000E124E96EFF0EE220EA6EED6607D02F0E41
:0E960000EF6404D03A0EEF6001D0F32A12009E
:02960E00FF0E4D
:10961000E350346E480E01D04C0EE76EE72EFED7B5
:0E962000E76AE72EFED7342EF7D700001200BF
:02962E00000E2C
:10963000F36E00EE00F00D0E01D81200EA6002D0C9
:0E964000EE6AFCD7F350E9601200EE6AFCD728
:02964E001CEE10
:1096500000F02CEE00F0F86A219C5AEC49F007EC7F
:0A96600000F05BEC45F0FBD71200B0
:06966A00FF0EE350ACBA54
:1096700004D0AF6AAB8EAC8A949CACA2FED7AD6E20
:06968000F36EF46A120013
:0A968600256A080EE76ED890293619
:1096900025362E50255C02E3256E292AE72EF7D7C2
:0296A0001200B6
:0E96A200303132333435363738396162636423
:0396B000656600EC
:0D96B300010207000000000000040000009C
:1096C000000000000000000000000000000000009A
:1096D000000000812D2D2D2D2D2D2D2D2D2D2D2DED
:1096E0002D2D2D2D2D000000000000000000000099
:1096F00000000000000000D9C6DE16364A44FE0015
:1097000000000000000000FFFFFFFFFF000000005E
:109710000066459A45BC45F2450C4670468C461697
:10972000475647A847D2474C488A48D048F2484055
:10973000499649EE49064A1C4A324A464A5C4ADE84
:079740004A004B204B4E4B89
:0997470000000000000000000019
:109750000000000000000000000000000000000009
:1097600000000000000000000000000000000000F9
:0C977000000000000000000000000000ED
:04977C0000000000E9
:1097800000000000000000000000000000000000D9
:10979000000000000000000000000000FF000000CA
:0197A00000C8
:0F97A10080000000000000000000000000000039
:1097B00000000000000000000000000000000000A9
:1097C0000000000000000000000000000000000099
:1097D0000000000000000000000000000000000089
:0197E0000088
:0497E1000000004D37
:020000040030CA
:0100010002FC
:0100020000FD
:0100030017E5
:0100050000FA
:010006008178
:010008000FE8
:01000900C036
:01000A000FE6
:01000B00E014
:01000C000FE4
:01000D0040B2
:0200000400F00A
:100000004E4F50484F4E45000000000000000000D9
:1000100000000000000000000000000000000000E0
:100020004F564D530000000000000000000000008B
:1000300000000000000000000000000000000000C0
:100040004B00000000000000000000000000000065
:1000500000000000000000000000000000000000A0
:100060000000000000000000000000000000000090
:100070000000000000000000000000000000000080
:100080000000000000000000000000000000000070
:00000001FF
